:020000040800F2
:10500000001C0020D5500008398C0008418300089E
:105010000000000000000000000000000000000090
:10502000000000000000000000000000899A000855
:10503000000000000000000009940008C59B000863
:10504000E7500008E7500008E7500008E750000864
:10505000E7500008FD5D0008E7500008E750000831
:1050600000000000E7500008255D0008E750000838
:10507000E75000082988000800000000E7500008F9
:1050800000000000E75000080000000000000000E1
:10509000E750000800000000E7500008E750000853
:1050A000E7500008E7500008E750000841A6000854
:1050B000E7500008E7500008000000000000000072
:1050C0000348854600F040FD00480047B5B9000898
:1050D000001C00200448804704480047FEE7FEE724
:1050E000FEE7FEE7FEE7FEE7619C0008C15000080E
:1050F00030B50B46014600202022012409E00D4670
:10510000D5409D4205D31D469540491B25469540F7
:1051100040191546521E002DF1DC30BDF0B51FB40C
:105120000646002082B005464024019100901BE015
:10513000019922460F46304600F0F0FB049A059B89
:10514000801A994110D310461946224600F0D6FB2A
:10515000361A8F410197224601200021009F00F05E
:10516000CDFB38184D4100902046641E0028DFDC3E
:10517000019B00982946324607B0F0BD03460B4319
:105180009B0703D009E008C9121F08C0042AFAD2FD
:1051900003E00B780370401C491C521EF9D2704783
:1051A000D2B201E00270401C491EFBD270470022BF
:1051B000F6E710B513460A4604461946FFF7F0FF16
:1051C000204610BD30B504460020034600E05B1CBD
:1051D000934203D2E05CCD5C401BF8D030BDF8B503
:1051E00002464A40D40F42004B0052085B089A42E4
:1051F00002D20246084611464A0023D0C30D4A0097
:10520000DDB2120EAD1A202D35DA49020126490A07
:10521000F6058A19002C00D0524220214F1B11465E
:10522000B9402A411018C20D9A4221D0002C17D043
:10523000012D08DCDA05801AD20F8019D207DBB203
:1052400000F098FBF8BDDA05801A012340001B0628
:10525000C01880185A428018CA0F1043490007E04E
:105260004908C2071143DA05801A801940088018DE
:1052700000F078FBF8BD61000122511A001BF7E72E
:105280000122D2075140AAE70122D2075040A6E7E7
:10529000024670B54A40D30FDB0740002DD04A00CC
:1052A0002AD0010E140E000212020919400A520AF5
:1052B0008418E50104465443000A120A2E045043A0
:1052C000A4194219200CC543AA18120C0125AD03DC
:1052D000521C521912047F39240400D0521C10436E
:1052E00001D44000491EC2B20C06C0092018401C5F
:1052F0004008802A02D003E0002070BD4008400032
:10530000002900DA0020184370BD70B502464A40FB
:10531000D50F40004A00ED0740085208002814D07D
:10532000002A12D0C40DD30D41020120C005520243
:10533000490A520AE41A091812187D34914201D31D
:10534000641C00E04900002C01DA002070BD00233D
:10535000914201D3891A0343400849000028F7D13C
:1053600000290AD0914202D10121C90705E09142EA
:1053700001D2012101E00121C943E005C018401913
:1053800000F0F0FA70BD420005D04200120E524209
:105390008A4201DB00207047C905081870470000E9
:1053A000F0B507460846584087B0C00F0490480043
:1053B0000E46590040084908BC1A884105D23846B3
:1053C00031461E4617460B46024658004008104319
:1053D0004CD0300D039040055900400D490D05900B
:1053E000401A0290402872DA18030121000B0905C7
:1053F0000843019004980092002805D00199524278
:105400000020884100920190029840210A1A0199D7
:10541000009800F073FA05460C466B4607CB00F087
:105420008EFAC0197141039A0E0D0023D71756400A
:105430001A467A40164344D0049A002A2DD0029A84
:10544000012A039A15DC1205C01A9141012636057E
:10545000001C7141D20F059ED20700930192029663
:105460002A46234600F0CCFA07B0F0BD3846314654
:10547000FAE71605224A0F46B218C01AB7410121B1
:105480000905001C4F4100187F4111461818794149
:10549000E20F10436D19644113E0E2076D081543F4
:1054A0006408C2071443039A01261205C01A9141E9
:1054B0003605001C7141CE07400830434908C0182A
:1054C00051412A46234600F08EFACDE7FFE70498C3
:1054D00001224000C117121A00238B410498314663
:1054E000C417381AA141EEE730B40124E407634041
:1054F00030BC55E730B40124E407614030BC4FE7CD
:105500000000E0FFF0B51FB488B00B9909980024A3
:1055100048400999C00F490049080991C0070B99F3
:105520000090490049080B9109990898A64608433C
:105530001CD00B990A98084318D009980124400000
:10554000420D4800410D099824050003000B20433B
:1055500009900B980003000B20430B9050181C4936
:105560004018002201901446104605E00020014634
:105570000DB0F0BD032801DA034600E003239C468A
:10558000C11A0AAE0AE05F0008ADED5B4F00F75BA1
:105590007D430027AA187C41491C5B1E6145F2DD52
:1055A000410004AB5A522104120C0A43240C401C43
:1055B0000828DFDB01980290009970460191009065
:1055C000059B049A0799069800F01AFAD0E70000A4
:1055D0000DFCFFFFF0B50C465C4085B0E40FE4071E
:1055E00003944C000026640859009446490802467A
:1055F0000296224321D062460A431ED06200570D14
:105600004A000E032303550D012402462C492405AC
:10561000781B1B0B360B4018234326436146009032
:105620001C46501AB44103D30098401C009002E07D
:10563000921800985B41002803DA0020014605B06B
:10564000F0BD0020012109050746864611E06446A9
:105650001D46141BB54106D36546521BB341744623
:1056600007430C43A646CD07400849082843921833
:105670005B4105460D43EAD11046184313D06046FE
:10568000194650407140084306D06046101AB34195
:1056900006D20122002306E000220123DB0702E0FC
:1056A0000122D2435310009874460105381C614111
:1056B000029C039D0019694100F095F9BFE70000C5
:1056C000FD03000070B54B005B0803430BD04B009B
:1056D0005C0D002633466542B341D417AD1AA34191
:1056E00002DB0020014670BD12053018514170BD2B
:1056F000C217C10F504010B54018CA0796230021A9
:1057000000F038F910BD10B500229623114600F0C4
:1057100031F910BD0EB5C217C10F5040CA0740186D
:105720000021054B0293019200910A460B4600F0BE
:1057300067F903B000BD0000330400000EB5054951
:105740000291002100910A460B46019100F058F9A0
:1057500003B000BD33040000C20F4100400201232A
:10576000400ADB05D207090EC0187F2901DA0020A4
:105770007047962903DC9623591AC84001E09639F0
:105780008840002AF4D04042704741004002012284
:10579000400AD205090E80187F2901DA00207047DF
:1057A000962903DC9622511AC840704796398840E2
:1057B0007047000070B5CD0F4A0009030123090BA3
:1057C0001B0519430B4BED070024520D9A4201DAD9
:1057D000002070BD074B34339A4203DC9A1A00F064
:1057E0009DF802E00449511888402C43F1D0404212
:1057F00070BD0000FF030000CDFBFFFF4A0009035E
:105800000123090B1B051943094B10B5520D9A4290
:1058100001DA002010BD064B34339A4203DC9A1A99
:1058200000F07CF810BD03495118884010BD0000FD
:10583000FF030000CDFBFFFFC20FD207400040086E
:105840000BD0C10D0723DB01C91840020905400A2E
:105850001143C208400711437047002001467047BA
:1058600010B5002904DB0124E40740428C412146A5
:10587000002B04DB1C460123DB075242A3418B4271
:1058800000D1824210BD000010B5002904DB0124C4
:10589000E40740428C412146002B04DB1C460123D7
:1058A000DB075242A341994200D1904210BD000053
:1058B000CB0FDB07490010B5490802460A4307D061
:1058C0000A0D07240903E401090B121B002A01DC5D
:1058D000002010BDC900440F0C43C100E018D205E0
:1058E000801800F03FF810BD0122D207002800DB2D
:1058F000101A002900DB511A8142704710B5202A86
:1059000004DB0146203A9140002010BD9140202345
:105910009C1A0346E3401943904010BD10B5202A5D
:1059200004DB0846203AD040002110BD0B46D3408E
:10593000D0402024A21A91400843194610BD10B54A
:10594000202A06DBCB170846203A1041C1170B432B
:1059500006E00B461341D0402024A21A9140084390
:10596000194610BD002904DA401C490001D1400845
:105970004000704770B40024050C05D110240004C9
:1059800002D1002921D01124050E01D100020834D2
:10599000050F01D10001241D850F01D18000A41C39
:1059A000002801DB4000641C002908D020252E1BA4
:1059B0000D46F540A14000D00121294308430106CE
:1059C0001B1B000ADB1D02D5002070BC7047DB05E5
:1059D000181880180029F8DA401C4900F5D170BC6D
:1059E00040084000704710B5002B08DA0024401C26
:1059F000614192185B411A4301D14008400010BD3B
:105A0000F0B51FB482B005460C0003D0084604F080
:105A1000CBFE02E004F0C8FE203002460090214692
:105A20002846FFF76BFF049B059A04460F46184370
:105A30001143084314D0184610431BD0009840214E
:105A40000A1A18460599FFF769FF05460E46009A9F
:105A500005990498FFF752FF084305D0012004E0A0
:105A60002046394607B0F0BD0020C11705430E435C
:105A70002C43374300990E986305401A7905E40AD0
:105A800000220C43FD0A0A3002D500200146E9E756
:105A90000105101969410C9C0D9D00196941FFF722
:105AA000A2FFDFE7FEB500231A461B1A8A4103DB7B
:105AB0000020014603B0F0BD4A000D0301212D0B6B
:105AC0000905520D0D43D10702D100186D41521E38
:105AD0005110FF31FF310131002704463E46384660
:105AE000009701910246012100200905FFF716FFEA
:105AF000C3197141F818324684468E464A416146C0
:105B00002846611A904104D36046241A954176468E
:105B10001F46241900986D41401C00903428E1DD97
:105B2000F91930467041091BA84103D20022D24323
:105B3000134601E00022134601980105381C71410B
:105B4000FFF751FFB6E70000064C0125064E05E0C1
:105B5000E36807CC2B430C3C98471034B442F7D38E
:105B6000FFF7B2FAA0C80008C0C8000870B58C18CA
:105B70000578401C6B075B0F01D10378401C2A118C
:105B800006D10278401C03E006780E70401C491CC8
:105B90005B1EF9D12B0705D40023521E0DD40B70C8
:105BA000491CFAE70378401CCB1A921C03E01D78CD
:105BB0000D70491C5B1C521EF9D5A142D8D30020A0
:105BC00070BD000038B50446064805490068FFF777
:105BD0008FFA604300E0401E00900028FBD138BDE2
:105BE00040420F0088010020F8B504460068816833
:105BF0008907890F012902D10168C90722D181686B
:105C0000114A10261140012500290ED1816829432F
:105C100081600120FFF7D6FF01F062F807460CE033
:105C200001F05EF8C01B0A2807D9606D304360653B
:105C3000A06D2843A0650120F8BD20680068C0431E
:105C4000C007EDD10020F8BD170000801FB50B483C
:105C500000900B4801900B4802900B480390694656
:105C60000A4805F097F90A4A08481146083905F02C
:105C70007FF800F0A9FA002004B010BDA9C6000802
:105C800085C60008E5C60008E3C6000894010020A8
:105C900010000020F8B51848808F00282AD0174C33
:105CA0000125E16AED051648A94201DB022100E069
:105CB0000021017000F0CAF90126F6020527A08232
:105CC0003F070FE00F4801F021FA80B2A083E18B7B
:105CD000421A032A01DC814204D9E0833146384666
:105CE00000F0B0F9E06AA842ECDA01223146384609
:105CF00000F0EFFFF8BD0000EC0D00203C0100209B
:105D0000840000200816002010B500231A4603E086
:105D1000845CE3189BB2521C8A42F9D3D84380B208
:105D200010BD000010B5034800F096FD024800F0D9
:105D300093FD10BD9C1700205417002030B5446C13
:105D40001C252C400125A540046C65600468636037
:105D50008368102B036803D099600068C26030BD6F
:105D60009A600068C16030BD1449012048720A463B
:105D700002205E32507203203C3A507204200E3AE8
:105D800050720F480D4B0078087022310870203196
:105D900008770C495A1C087858714978997123334F
:105DA00018715971203318775977107551751A4643
:105DB0001E3210755175107651767047EC11002027
:105DC0003E0100206401002010B503F033FE2020C6
:105DD00003F0EEFE012005F047FB002003F0E8FE93
:105DE000044805F0E5F9044805F094FC002005F0AE
:105DF000C9FC10BD0001002083800000F8B503F04D
:105E0000E5FE05200121000700F056FF0025144C97
:105E1000002800D06560134E0221304600F04CFF90
:105E2000002815D1012020700F48808F00280ED047
:105E30000127BF0200223946304600F04AFF0A20FF
:105E400004F006FF01223946304600F042FF65604B
:105E5000012000F069FE022000F066FEF8BD00009F
:105E60007401002000040050EC0D00207047000079
:105E700010B5084900224A6107494B684C15234375
:105E80004B604B68082423434B60C009C00102608B
:105E900010BD0000E4170020002002407FB500255F
:105EA0000C460646039500F00FFEE009029003A998
:105EB00001960095684600F09FFD002804D000F090
:105EC000D7FD002004B070BD00F0D2FD0120F9E73D
:105ED00010B5002302E0C45CCC545B1C9342FAD39F
:105EE00010BD000010B5214A00219069C30520486B
:105EF00004D54169022319434161911593699B05BA
:105F000005D543690124234343616302194393691F
:105F10005B0505D54369082423434361E301194325
:105F200093691B0505D54369042423434361630238
:105F3000194393699B0405D54369102423434361A6
:105F40006302194393699B0304D5446920231C43CE
:105F5000446119439369DB0305D543694024234316
:105F60004361A0020143916110BD00000020024086
:105F7000E417002070B5054600F0B2FE0646184C46
:105F80000AE0681C08D0002D04D000F0A9FE801B98
:105F9000A84201D9032070BDA069C007F1D1A06952
:105FA000800701D50220A061A069C00511D4A069B5
:105FB00080050ED4A06940050BD4A069000508D463
:105FC000A069800405D4A069800302D4A069C0033D
:105FD00003D5FFF787FF012070BD002070BD0000D2
:105FE00000200240F8B51746002605460C4600F092
:105FF0006BFD09E029460220226800F047FD0028D9
:1060000004D1241D2D1D361DBE42F3D300F030FDFA
:10601000BE4201D20020F8BD0120F8BD10B50849EC
:1060200002460020054B497905E044001C5B944280
:1060300003D0401CC0B28842F7D310BD901300209B
:106040007000002010B500F03CFE10BD10B50948EE
:1060500001F05CF880B2FFF771FB074A074BFFF7CE
:1060600051FA0022064BFFF7B5FAFFF7C7FB80B2E3
:1060700010BD000008160020F853E3A59B843E40A5
:1060800000408F4070B50024204603F055F9474981
:106090004748A200641CE4B28150142CF9D346494D
:1060A00044480A7902754979417544490A7802766B
:1060B000497841763F490520133148720A2005F09E
:1060C00019FB7D20400105F02FFB3A4900221331D6
:1060D0000C2005F0F9FB00210C2005F007FC3848E6
:1060E00001F014F8344C0125223C2085AD0309E071
:1060F000334801F00BF880B22085E18EFF392D394D
:10610000884206DBE18E80B28842F1D34919884289
:10611000EED8022005F03EFB002003F00DF9294DDA
:1061200000210F2005F066FA28422064F8D0206C88
:10613000411C38D0400435D58122D20100210F20E6
:1061400005F097FB0021102005F054FA410619488C
:10615000490E0022C73005F083FA164DC735687A1C
:1061600005281FD102221549681DFFF72BF80028CA
:1061700018D11148AE7C66710422691C3630FEF7D6
:10618000FDFF29461331084672000D466930FEF7BF
:10619000F5FF60792946420005484838FEF7EEFFD2
:1061A0000320207070BD04F073FB0000FFFF0100AE
:1061B000F01300204D120020920000206401002006
:1061C0000816002000D0272410B5144C144822468D
:1061D00010321146083904F0CBFD0022114BE16862
:1061E000A068FFF7F7F9104A104B05F0EDFC00220C
:1061F0000F4BFFF77FF900220E4BFFF783F9FFF7F4
:1062000057FB206000221346E168A068FFF728FBD7
:1062100001D0206810BD0020206010BD00000020CB
:106220009401002000AA8F406C45D9CC955BC83FF3
:106230000000F03F40A5E54010B5084800F096FA90
:106240000A21064800F032FA044800F01DF98005E2
:1062500003D5024800F01AF980B210BDAC15002039
:10626000F8B52F4D00220121284600F032FDFFF73E
:10627000E3FFFFF748FA2B4E3146FFF746F82A4C6A
:106280000122A0601146284600F023FD2749A0689E
:10629000002588423EDB2078254F002815D0257048
:1062A000FFF7CAFFFFF72FFA3146FFF72EF8A0607D
:1062B000FFF7C2FA00223B46FFF716F900221D4BFA
:1062C000FFF720F9FFF7F4FA6060A068FFF7B4FA6F
:1062D00000223B46FFF708F9174A184BFFF712F95F
:1062E00006460F466068FFF7A7FA134A144B52425E
:1062F000FFF708F932463B46FFF752F8FFF7D8FAA6
:1063000010496060884201DD616004E0FF21C90539
:10631000C84200D365606068FFF737FAC0B2F8BDC5
:106320000004005000401B44480000200000604072
:1063300000000C4000E064403333333333B330406B
:10634000CCCCEC3F0000C842F8B5054604464035C9
:10635000287C0026012808D0012028742068816844
:106360008907890F01290ED101E00220F8BD0168DB
:10637000C90708D0606D2021084360650126002010
:1063800028743046F8BD616DFF220132914302222C
:1063900011436165C1688907890F0091C168890847
:1063A0008900C1602068816892071143816000F014
:1063B00097FC07460EE000F093FCC01B0A2809D9A1
:1063C000606D022188431021084360650020287415
:1063D0000120F8BD206880680028ECDB2068C168D7
:1063E000009A1143C160606D80088000401C6065A8
:1063F000C5E70000F8B506460D464036317C012958
:106400000DD00121317401688A68520709D5416DA8
:10641000202211434165002030740120F8BD022084
:10642000F8BD174B6A68D80547109A42154C8A6A1E
:106430002B6812D05B035B0B1A438A6229684903FD
:1064400005D5A1680143A1600A20FFF7BBFB2868BE
:10645000800312D5A06838430EE05B035B0B9A43C0
:106460008A622968490302D5A1688143A16028682E
:10647000800302D5A068B843A06000203074F8BD46
:106480000110000000270140406D70470068006C5B
:106490007047000070B5040006D0606D26460025E8
:1064A0004036002802D006E0012070BDA565357495
:1064B000204600F0D3F8606DC00603D421688868D8
:1064C000400705D5606D1021084360653574EBE722
:1064D000606DFF220132904302221043606588689C
:1064E0008207920F5B48012A02D10A68D2072BD19A
:1064F000032362689B079A4205D05B429A4202D00E
:106500005B009A4209D10A69920092080A612168E7
:106510000A6963681A430A610CE00A6992009208EA
:106520000A6181680F2292049143816081686268E8
:10653000114381602168CA6818239A43CA602168A0
:10654000CA68A3681A43CA6081680122520691434F
:1065500081608168A28E5206114381602068816843
:10656000C90004D4816801221207114381602068A8
:10657000C168394A1140C1602069E168022825D00C
:1065800000200143204620300278037B52035B0049
:106590001A431143226B1143A26992031143E2692A
:1065A000D20311432268D3681943D160616A0A4655
:1065B000FF3AC23A05D0A26A11432268D368194350
:1065C000D16042780121012A02D00BE00420D8E7F3
:1065D0000078002823D0606D202210436065A06DF4
:1065E0000843A065E06B012820681FD00169C90736
:1065F00003D0016949084900016120684169C9085F
:10660000C900416120684169A26B11434161A565E0
:10661000606D80088000401C6065002070BD2068AF
:10662000C26801231B041A43C260DBE70269FF232F
:106630009B009A43026120680269236CA66C1A438E
:10664000636C33431A430261206802690A430261A2
:10665000D3E70000002701401902FEFF10B586B005
:10666000044614216846FEF7A2FD0E4920688842C0
:1066700016D10D48416B421511434163C16A012295
:106680001143C162C06A6946104005900220009023
:1066900003200190002002900520000700F050FA2E
:1066A00006B010BD0024014000100240F8B50446B9
:1066B0004069254640350E4608280BD02068C06842
:1066C000C00709D0606D2021084360650020287450
:1066D0000120F8BD082700E00C2700F001FB009026
:1066E00011E0701C0FD0002E05D000F0F9FA0099CF
:1066F000401AB04207D9606D04210843606500204C
:1067000028740320F8BD206800683842E9D0606D25
:1067100001214902084360652068C16809058A0FA4
:106720000C21002A1BD12022125D002A17D10268F9
:10673000120714D5826853070122002B08DB436837
:106740008B434360606D130298431043606506E01D
:10675000606D202318436065A06D1043A065A0699B
:10676000002801D1206801600020F8BD70B5044602
:10677000216800208968490721D425464035297CB5
:1067800001291CD001212974E169012904D0204686
:10679000FFF72AFA002811D1616D0A4A1140FF2241
:1067A0000132114361650021A165297422681C2111
:1067B000116021688A6804231A438A6070BD022030
:1067C00070BD0000FEF1FFFF30B5014620314A796F
:1067D0000023022A04D00422C2630B71012030BDC1
:1067E000026814680E25AC431460026814686408DB
:1067F00064001460446C1C22144001221546006C95
:10680000A54045604A7118460B7130BD70B5002433
:10681000014620314A79022A03D00421C1630124B0
:1068200018E0026813680E25AB4313600268136812
:106830005B085B001360436C1C2213400122154669
:106840009D40036C5D604A7100220A71816B0029D2
:1068500000D08847204670BDF0B4016C0D68016817
:106860000C68466C1C2304221E401746B7402F427A
:106870000ED067070CD50C68A40602D40C689443AC
:106880000C60416C19408A40016C4A60016B1AE04F
:106890000227B74002462F402032002F17D0A7070B
:1068A00015D50C68A40605D40C680A25AC430C6009
:1068B00001215171446C02211C40036CA1405960BC
:1068C00000211171C16A002918D0F0BC08470827BF
:1068D000B7402F4212D0240710D50C680E25AC43C8
:1068E0000C60446C01211C400B46A340046C6360A7
:1068F000C163517100211171416BE4E7F0BC704735
:1069000070B504003CD01F48256814212818FEF7F4
:10691000EFFB800060641C48206402212046203088
:106920000246417129681948E3680140A068666918
:106930001843236933431843A3691843E369184391
:10694000236A1843084328600121A068890388420C
:1069500010D00D488030836A656C1C210D400F26D5
:10696000AE40B3438362656C63680D40816AAB409F
:106970000B4383620020E06301215171107170BDEF
:10698000012070BDF8FFFDBF000002400F80FFFF37
:10699000F8B504468C46203001790025012909D03C
:1069A0000126067141790027012905D007710225CA
:1069B0002846F8BD0220F8BD02214171E763206836
:1069C000016849084900016061462046FFF7B6F9B1
:1069D000206B00282068016801D00E2205E0042207
:1069E00091430160206801680A2211430160206818
:1069F000016831430160DBE7F8B51A4E0546307C8B
:106A00000F46012807D0012030741748FFF7B2FA6B
:106A1000010002D021E00220F8BD0020C043386010
:106A20006C6814E02046FFF723FA0F48FFF7A2FA3C
:106A300001460E48426808239A4342604268431563
:106A40009A434260002901D03C6006E08034A86887
:106A50006A68C0018018A042E4D80020307408465B
:106A6000F8BD0000E417002050C3000000200240E1
:106A700005484168022211434160416801221143E7
:106A8000416000207047000000200240F8B50C4C27
:106A90001646207C0F46012808D0012020740948A2
:106AA000FFF768FA0025002802D006E00220F8BDB2
:106AB00065613E600348FFF75DFA2574F8BD00008C
:106AC000E417002050C3000011484168C9070BD0EB
:106AD000EFF3108172B60F4AC2600F4AC26081F3B1
:106AE00010884168C9070ED1416889070DD5EFF3B9
:106AF000108172B6094A0261094A026181F3108865
:106B00004068800701D501207047002070470000D1
:106B100000200240EFCDAB8905040302BFAE9D8C7F
:106B2000161514137047000010B504494A69024253
:106B300002D04861FFF7F6FF10BD000000040140DD
:106B4000FCB500230124A2E027462A469F403A4094
:106B50006FD04D68012D05D0022D03D0112D01D02D
:106B6000122D16D185680326AC465D00AE46AE40B8
:106B70006546B543AC46CE687546AE4065462E4385
:106B8000866046680D79BE43ED06ED0F9D403543A6
:106B90004560C6685F000325BD40AE46AE4335463E
:106BA0008E68BE402E43C6604E68022E01D0122E63
:106BB00014D1DE08B60036180196366A5D07B44671
:106BC000EE0E0F25B54000966646AE43B4460D69FD
:106BD000009EB54066462E43019D2E6206687546AE
:106BE000AE430D79AD07AD0FBD40354305604D682F
:106BF000ED004BD5294D6E6B26436E639E08284DE4
:106C0000B6007519AC46AD689E07360F0F27B74022
:106C1000BD4305273F07B84201D1002715E0214FAA
:106C2000B84201D1012710E01F4FB84202D102271C
:106C30000BE02BE01D4FB84201D1032705E01C4FAC
:106C4000B84201D1052700E00627B7402F4365462B
:106C5000AF60184D2E684F689643FF0300D516436A
:106C60002E606E684F689643BF0300D516436E6072
:106C7000AE684F689643FF0200D51643AE60EE68DB
:106C80004F689643BF0200D51643EE605B1C0A684E
:106C90001546DA4000D057E7FCBD00000010024066
:106CA000000001400004005000080050000C00509B
:106CB000001C0050000401400069084000D0012081
:106CC0007047426913460B401B0491430B43836199
:106CD0007047002A01D081617047816270470000CF
:106CE00001488068704700007C01002002488168EC
:106CF00002788918816070477C01002010B508482F
:106D000000240168402211430160204600F00AF887
:106D1000002801D0012401E000F042FA204610BD15
:106D20000020024070B504460D4D7D202978C0003A
:106D3000FEF7DEF901460B480068FEF7D9F900F0CE
:106D40002BFF002809D1042C07D200222146401E27
:106D500000F04EFA00206C6070BD012070BD000094
:106D60007C0100208801002070477047F8B502F0D0
:106D70002DFF604C0120E070208AFEF7C4FC014624
:106D80007F20C005FEF7C1FA5B4D06462968FEF775
:106D900026FA28600120E16AC005814201DA08462E
:106DA00003E03046FEF770FAE062FF21C9050025D6
:106DB000C84200D3E562607800280BD102214F4819
:106DC000FFF77AFF02004E494E4817D00022FFF726
:106DD00080FF256302214948FFF76EFF4A4E0028D5
:106DE00055D02563B08AFEF78EFC434F3968FEF715
:106DF0007BFD5FD24549012008705DE00122D1038F
:106E00004048FFF766FF208AFEF77DFC01467F20A1
:106E1000C005FEF77AFA216BFEF7E1F93C492063E1
:106E20008842D7DD38480127F926403000900A21F2
:106E30003046FEF75DF9002903D131493148FFF7AB
:106E400001F902212D48FFF737FF002801D0002764
:106E500001E0002F12D102212848FFF72DFF002862
:106E60000CD104F079FE00990120888005F0D0FB58
:106E7000642003F0EDFE28492648C8600A2003F08C
:106E8000E7FE3046761EF6B20028D0D1A2E7208A6F
:106E9000FEF739FC01467F20C005FEF736FA216B6C
:106EA000FEF79DF91D49206388429BDB1A4919486A
:106EB000C86097E715480570708F401EFEF718FCF4
:106EC0003968FEF711FD06D82079002803D014494F
:106ED0000120087001E012480570708FFEF713FC66
:106EE0003968FEF701FD04D22079002801D004F0B2
:106EF000F7FDF8BD3C01002078010020000400509F
:106F00000080000000000050EC0D00207600002002
:106F1000000040400400FA0500ED00E00000A04041
:106F200086000020704770B5040010D0022025466E
:106F30002035A873204601F07FFCA87B032805D0EC
:106F4000204600F0B9F80020A873687370BD0120D6
:106F500070BD7047704710B5044600680168C943AA
:106F6000C90708D18168C943C90704D1012141601B
:106F70002046FFF7FBFE20680168C943890708D453
:106F80008168C943890704D4022141602046FFF784
:106F9000EBFE20680168C943490708D48168C943EA
:106FA000490704D404214160204600F0F7F8206826
:106FB0000168C943090708D48168C943090704D493
:106FC000082141602046FFF7ADFF20680168C943F2
:106FD000C90608D48168C943C90604D41021416098
:106FE0002046FFF7C2FE20680168C943890608D41D
:106FF0008168C943890604D4202141602046FFF7F7
:10700000A9FF20680168C943490608D48168C943BB
:10701000490604D4402141602046FFF79AFF10BD85
:10702000F8B5040005D025462035A87B002802D0FD
:1070300006E00120F8BD00206873204600F04EF8FD
:107040000220A8732068C26884466368012B01D1BE
:107050000620824316486169814202D0072040031E
:107060008243002B01D1D82082431248A6680240F7
:1070700018463043676A266A3E433043A66A304367
:107080001043002B02D0012B04D005E02369E269F4
:107090001A4300E0E2681043054A914202D0A26917
:1070A000114308436146C8600120A8730020F8BD61
:1070B000FFFF0000F8F119FF10B50068054988428C
:1070C00007D10548816B4900490881630D2000F014
:1070D00073F810BD007C00400010024010B500683D
:1070E000084988420CD10848816BC204114381636E
:1070F000002201210D2000F07BF80D2000F06CF83B
:1071000010BD0000007C0040001002400068C06913
:1071100070470000F8B50446022025462035174682
:10712000A8731D480268C3041A4302602068C2683D
:107130009B121A43C2602068026901263243026131
:10714000226810205060206881611021204601F0E3
:10715000E3FB03281FD021680820486020684761AE
:107160000821204601F0D8FB032814D0204601F066
:1071700063FBA87B03280ED02068816831438160BF
:1071800020680169314301612068016904221143CB
:107190000161AE730020F8BD00040140704700009B
:1071A0000448416B012211434163816B0204114386
:1071B0008163704700100240002809DBC106C90E38
:1071C0000120884003490860BFF34F8FBFF36F8FE2
:1071D0007047000080E100E0002805DBC106C90E11
:1071E00001208840014908607047000000E100E08C
:1071F00010B503F02BFB10BD02494A6882434A6078
:107200007047000000700040024801688215114379
:10721000016070470070004002494A6802434A60BA
:1072200070470000007000400548016802221143C9
:1072300001600448016904221143016130BF7047B5
:107240000070004000ED00E0F0B5154A1368154DE0
:1072500054152D6A2340ED07ED0F002B04D0002DAF
:1072600002D01668A64316601668B608B600064334
:1072700016600D48076904263743076101290DD0C0
:1072800040BF20BF20BF0169B1430161002B04D082
:10729000002D02D0106820431060F0BD30BFF2E72F
:1072A000007000400000014000ED00E0F8B5044629
:1072B00000780027534D800671D5524E403EB06B8A
:1072C000C00004D4B06BA9050843B06301274E4841
:1072D0000168C90511D40168821511430160FFF7E7
:1072E000FFFC009005E0FFF7FBFC0099401A6428C2
:1072F00037D845480068C005F5D53268032109052F
:1073000060680A400140914208D08103890F032937
:1073100004D13168890301D50120F8BD2A69032110
:1073200009040A4022D0084090421FD020788006ED
:107330001CD528692A6988430121C9040A432A61A6
:107340002A698A432A612861C0050FD5FFF7C8FC66
:10735000009008E0FFF7C4FC0099411A2B488142D5
:1073600001D90320F8BD28698005F3D56168880339
:10737000800F032805D132680005824301400A438B
:1073800032602869032261681204114008432861B1
:10739000002F04D0B16B012000078143B163207836
:1073A000C00705D0E868A168800880000843E8604D
:1073B0002078800705D5E8680C218843E1680843F8
:1073C000E8602078400706D5E868032189028843F1
:1073D00021690843E8602078000706D5E8680321A2
:1073E0000903884361690843E8602078000606D5F0
:1073F000E868032189048843A1690843E860002004
:10740000F8BD0000401002400070004088130000EA
:10741000F8B50E46050038D05E480068C007C00FBA
:10742000B04214D25B4C20684008400030432060DA
:10743000FFF756FC074605E0FFF752FCC11B564814
:1074400081427AD82068C007C00FB042F4D12878B2
:10745000524C800705D5E068F0218843A9680843AD
:10746000E0602878C00752D06868022806D0032858
:1074700007D0216801280AD0890504E02168890322
:1074800001E021688901002903DB0120F8BD4907DB
:10749000F9E7E168890889000143E160FFF720FC12
:1074A0000746686802280AD0032814D001281ED095
:1074B00029E0FFF715FCC11B374881423DD8E06841
:1074C0000007800F0228F4D121E0FFF709FCC11B5F
:1074D0003148814231D8E0680007800F0328F4D199
:1074E00015E0FFF7FDFBC11B2B48814225D8E06862
:1074F0000007800F0128F4D109E0FFF7F1FBC11B61
:107500002548814219D8E0680007800FF5D121484D
:107510000168C907C90FB14217D901684908490074
:1075200031430160FFF7DCFB074608E005E0FFF7A9
:10753000D7FBC11B1848814201D90320F8BD15486B
:107540000068C007C00FB042F1D12878400706D5C7
:10755000E068072109028843E9680843E060287869
:10756000000707D5E0680721C90288432969C900D7
:107570000843E06000F03AF8E168094A0906090F9B
:10758000515CC8400749086007480068FFF7CAFB1C
:10759000F8BD0000002002408813000000100240E7
:1075A000EAC700088801002080010020044805493E
:1075B0000068C968044A4905490F515CC8407047D2
:1075C000880100200010024003C800080448054953
:1075D0000068C968044A8904490F515CC840704773
:1075E000880100200010024003C8000870B51A4A44
:1075F000D3681A490C2018408D0004280CD04E0086
:10760000082810D00C2810D050680004410F012029
:10761000C003491C884070BD1068C00601D50846EB
:1076200070BD284670BD304670BD98020C4C000FEE
:10763000205C1B029C0FD368641CDB0301D5314620
:1076400003E01268D20600D4294603F0C4F82246AB
:107650000023FDF763FD70BD0010024000093D00EE
:10766000FAC70008FEB505007ED0FE4CE7680C2086
:10767000E66807400120000406402878C00747D08C
:10768000082F05D00C2F0AD101200004864206D114
:10769000206880033CD568680028E5D038E00120E8
:1076A00069680004814203D121680143216011E02F
:1076B000052301221B0492049942216802D111433F
:1076C0002160F1E781432160216801400091206839
:1076D00090432060686800280DD0FFF701FB009000
:1076E00005E0FFF7FDFA0099401A64287BD820686E
:1076F0008003F6D50CE0FFF7F3FA009005E0FFF702
:10770000EFFA0099401A6428F0D820688003F6D474
:107710002878800756D50923E868042F0DD00C2F50
:1077200001D1002E09D000283CD0216899430143A3
:107730002160FFF7D5FA064628E02168490701D500
:10774000002891D061681F22120291432A69120217
:10775000114361602168994301432160FFF746FFAF
:10776000E16809060A0F00E08BE1BF49895CC84067
:10777000BE490860BE480068FFF7D4FA002873D1FC
:1077800020E0FFF7ADFA801B0228AFD82068400741
:10779000F7D560681F210902884329690902084357
:1077A00060600FE02068400840002060FFF798FA12
:1077B000064604E0FFF794FA801B022896D820685A
:1077C0004007F7D42878C00660D5002F0CD0A869F0
:1077D00000284AD02068FF21013108432060FFF7CC
:1077E0007FFA06462EE0C1E02068800502D5A86930
:1077F0000028A6D06068072149038843296A084306
:1078000060606068297F0002000A09060843606022
:10781000286A410B0120C003491C8840E168090621
:107820000A0F9149895CC8409049086090480068F7
:10783000FFF778FA002817D128E0FFF751FA801BEC
:107840000228A2D820688005F7D56068072149037F
:107850008843296A084360606068297F0002000A43
:1078600009060843606011E0E2E02168FF20013072
:1078700081432160FFF734FA064604E0FFF730FA4F
:10788000801B022872D820688005F7D42878794EAA
:10789000000724D568690028306910D00121084309
:1078A0003061FFF71DFA009005E0FFF719FA009923
:1078B000401A02285AD830698007F6D50FE04008F0
:1078C00040003061FFF70CFA009005E0FFF708FA7E
:1078D0000099401A022849D830698007F6D42878E0
:1078E000400766D500200290A06BC00006D4A06BB4
:1078F000012109070843A063012002905E48016846
:10790000C90511D40168821511430160FFF7E8F938
:10791000009005E0FFF7E4F90099401A642825D8A3
:1079200055480068C005F5D5FF20AA68013082429D
:1079300003D131690143316111E001218902002A3B
:1079400007D005231B029A4203D132690A433261F0
:10795000EFE7326982433261306988433061A86859
:10796000002810D0FFF7BCF9009008E05FE0FFF7B7
:10797000B7F901460098091A4048814257D8306942
:107980008005F4D50DE0FFF7ABF9009006E0FFF7B6
:10799000A7F90099411A3948814248D830698005D1
:1079A000F5D40298002804D0A06B01210907884370
:1079B000A063686A002866D00C2F3ED001263606E8
:1079C0000228206805D0B0432060FFF789F90546FA
:1079D0002FE0B0432060FFF783F9074604E0FFF78C
:1079E0007FF9C01B022822D820688001F7D4E96AF9
:1079F000A86AE2680843296BFD231B049A431143DC
:107A00000843E060206830432060FFF769F90546CD
:107A100004E0FFF765F9401B022808D820688001C0
:107A2000F7D530E0FFF75CF9401B022801D90320AD
:107A3000FEBD20688001F5D425E00128F8D0E0687B
:107A400001210904AA6A014091421AD10F21890437
:107A5000EA6A0140914214D1032189050840296B4B
:107A600088420DE000100240EAC7000888010020AB
:107A70008001002040100240007000408813000088
:107A800001D00120FEBD0020FEBDF8B504000ED0DF
:107A9000FF27606A0537002500280AD02561656147
:107AA00026464036A562707C002807D00AE00120F7
:107AB000F8BD6068B842F3D0E561F1E7357420465F
:107AC00000F03EF8022171742068026840239A4356
:107AD00002602123A26860689B021A40384010436C
:107AE000E3688A021340184323690B40217D184341
:107AF000C907C90F0843A169931019400843E169F8
:107B0000382319400843216A802319400843A16A99
:107B100093001940084321680860A0690421000C03
:107B20000840616A102319400843216848602068B2
:107B3000C1699143C1616565012070740020F8BD81
:107B400010B586B0044614216846FDF730FB104995
:107B50002068884219D10F48416B82141143416358
:107B6000C16A01221143C162C06A00211040059020
:107B7000E0200090022001900320039002910491E4
:107B8000052069460007FEF7DBFF06B010BD0000C8
:107B90000030014000100240094910B5401E8842E3
:107BA00001D9012010BD074C60610321081F02F0BC
:107BB0004DFE0020A06107202061002010BD0000C4
:107BC000FFFFFF0000E000E0F0B502462032137E28
:107BD000012B1ED0012515760223537606687468A2
:107BE000B3687027BC430F68274377600068AC0711
:107BF000A04205D0084CA04202D0084CA04204D1BB
:107C000080244968A343194381605576002010768B
:107C1000F0BD0220F0BD000000080140001401404A
:107C200070B5050005D02C462034607E002802D0B7
:107C300006E0012070BD00202076284600F010F8F4
:107C400002206076291D286802F036F80120A0770E
:107C5000A076E076207760776076002070BD000027
:107C6000006801218907884204D10348816B012201
:107C7000114381637047000000100240F8B50546CB
:107C800004462035287E012817D001262E760220B2
:107C90006876226890687727FF23B8431B029843D1
:107CA00090600A68502A31D00EDC202A4BD006DCC6
:107CB000002A48D0102A3AD145E00220F8BD302AE7
:107CC00041D0402A33D136E0602A27D0702A12D022
:107CD00001200003121A2AD0824228D1CB684A68B8
:107CE0008968206802F014F82068816801229203F4
:107CF000114381601BE0CB684A688968206802F004
:107D000007F8216888683843886010E0CA684968C5
:107D1000206802F077F85021206806E0CA684968B8
:107D2000206802F080F86021206801F0FCFF6E7688
:107D300000202876F8BDCA684968206802F062F819
:107D400040212068F1E711462068EEE710B586B0C3
:107D5000044614216846FDF72AFA012120688907A4
:107D6000884212D10A49CA6A02200243CA62C96A19
:107D7000019001400591410200910021029103917F
:107D8000049069460348FEF7DBFE06B010BD000014
:107D90000010024000040050F8B5064604462036A4
:107DA000307E0D4601280BD0012008273076002AAE
:107DB00008D0042A16D0082A2AD00C2A4DD137E040
:107DC0000220F8BD206801F0B6FF206881693943C0
:107DD0008161206881690422914381612068816901
:107DE000EA6812E0206801F0BEFF20688169012284
:107DF000D2021143816120688269012189028A438C
:107E0000826120688169EA6812021143816124E07D
:107E1000206801F0C1FF2068C1693943C161206851
:107E2000C16904229143C1612068C169EA6812E016
:107E3000206801F0CCFF2068C1690122D202114301
:107E4000C1612068C269012189028A43C261206838
:107E5000C169EA6812021143C16100203076F8BDA1
:107E600070B5050005D02C462034607E002802D075
:107E700006E0012070BD00202076284600F00FF8B3
:107E800002206076291D286801F016FF0120A077E6
:107E9000A076E076207760776076002070BD70472E
:107EA0007047704770470000F8B502680446D06913
:107EB00011689668814B05461D402023002D6CD02B
:107EC000F7077F4DFF0FBC460D402F4379D0254665
:107ED000C7078035002F06D0CF0504D501271762CC
:107EE0002A683A432A60820708D5F20706D0276835
:107EF00002223A622A6804273A432A60420708D5D8
:107F0000F20706D02668042232622A68022632432B
:107F10002A6002070AD50A461A406646324305D04F
:107F20002668082232622E6816432E60020508D5A4
:107F30004A0106D501222668D20232622A681A4313
:107F40002A602A68002A30D0800606D5880604D523
:107F5000616E002901D02046884728682168896819
:107F6000490602D42821084225D0204602F07FF994
:107F700020688168490619D5826840218A43826059
:107F8000206F002812D04F498163206FFEF73EFC1E
:107F900000280AD0206F816B06E0850611D58D067A
:107FA0000FD5616E77E020468847F8BD2046FFF781
:107FB00079FFF8BD05E02046FFF774FF0020286038
:107FC000F7E7256E012D56D1C50654D5CD0652D5FD
:107FD000102616622068816825464906403500292A
:107FE0002ADA226F116849680904090CE1D02F8B45
:107FF0008F42DED9698311680968890617D4016840
:10800000320191430160206881684908490081601C
:1080100020688168402291438160E36700202066E8
:1080200020680168B1430160206FFEF7CDFB288B0B
:10803000698B401A81B21AE0298B6A8B891A6A8B84
:1080400089B2002AB5D00029B3D00268FF252135B6
:10805000AA43026020688268520852008260E36787
:1080600000202066606620680268B24302602046F5
:10807000FFF716FF9DE7C50208D5750206D501205A
:10808000000510622046FFF70CFF92E7050605D5B4
:108090000D0603D5A16E002985D18AE7400688D553
:1080A000480686D5116820464024A14311608367A5
:1080B0000021816600F043F97BE700000F08000013
:1080C0002001000495A1000810B5040003D0A06FA2
:1080D000002802D007E0012010BD002174200155C6
:1080E000204600F027F82420A0672068016849088E
:1080F00049000160204602F00DF90128ECD0606AC9
:10810000002802D0204601F02FFF20684168092294
:10811000D20291434160206881682A2291438160A4
:1081200020680168012211430160204601F082FFAE
:1081300010BD0000F0B587B0064614216846FDF773
:1081400036F82C493068884251D12B48416B0122C6
:10815000920311434163C16A01221143C162C06AA3
:1081600000251040059003204002009002200327C4
:1081700001A9A1C104200490052069460007FEF76B
:10818000DFFC1F4C1D48A560E56081C48027E560C9
:10819000A7602020256160610002A0611848083CAA
:1081A000FEF7AEFB002801D0FDF760FE3467A66243
:1081B000144C1248214614382060032060601020BF
:1081C0000831A1C16561A561E56120462562FEF720
:1081D00097FB002801D0FDF749FEF466002201213B
:1081E0001B20A662FFF704F81B20FEF7F5FF07B07F
:1081F000F0BD000000380140001002403000024095
:10820000541700209C17002070B5C36F202B27D176
:1082100000290BD0002A09D0012483682403A3423B
:1082200006D10369002B03D1CB0701D0012070BD1B
:10823000034660331C7D012C12D001241C750023E1
:108240000366084C0368A34207D05C68240204D587
:108250001C680125AD062C431C6002F05BF970BD63
:10826000022070BD0048004070477047FFB50446CB
:10827000806F83B017460D4620285ED1002D0AD0AE
:10828000002F08D0A168C001814207D120690028D1
:1082900004D1E80702D0012007B0F0BD20466030CD
:1082A0000090007D012848D0009801210175002030
:1082B000802108512120A067FEF712FD2646403696
:1082C0000190378277820120A1680003814202D1A8
:1082D0002069002805D02F46002500990020087548
:1082E00011E00027F9E700228021204602F058F92A
:1082F000002815D1002F15D02168387888627F1C9E
:10830000708A401E7082708A019B00280698009037
:10831000E9D100224021204602F042F9002808D08D
:108320000320B9E728882168C005C00D8862AD1C0C
:10833000E6E72020A0670020AEE70220ACE7704708
:10834000034D044C04A002F025FAE560FAE70000B2
:108350000400FA0500ED00E0486172644661756C46
:10836000745F48616E646C65722E0D0A0000000037
:1083700070B586B014216846FCF719FF1248012435
:10838000C188012902D0022900D0C480C0880F49C9
:108390000128488305D0022801D100F0E7FB06B090
:1083A00070BD01220526D502360729463046FEF764
:1083B00090FC00210291039100950194694630469A
:1083C000FEF7BEFBEBE700002C0E00203C01002076
:1083D00070B501240E4DA403002221462846FEF765
:1083E00078FC002204212846FEF773FC0A2002F0E4
:1083F00036FC012221462846FEF76BFC0A2002F0DB
:108400002EFC002221462846FEF763FC70BD0000CA
:108410000004005070B501240E4DA4030022214633
:108420002846FEF756FC012204212846FEF751FC9F
:108430000A2002F014FC012221462846FEF749FCDE
:108440000A2002F00CFC002221462846FEF741FCDF
:1084500070BD000000040050F1B500240126154F46
:108460002546B603002231463846FEF732FC0A2084
:1084700002F0F5FB012231463846FEF72AFC600681
:10848000040E04213846FEF717FC002801D0641CB6
:10849000E4B2052002F0E3FB6D1CEDB2082DE1D340
:1084A0000098002803D0FFF793FF2046F8BDFFF7A0
:1084B000B1FFFAE700040050F8B50126154F054654
:1084C000B603002231463846FEF703FC0024E809D3
:1084D00001D0012200E0002204213846FEF7F9FB1A
:1084E0006806050E0A2002F0BAFB01223146384622
:1084F000FEF7EFFB0A2002F0B2FB002231463846BD
:10850000FEF7E7FB0A2002F0AAFB641CE4B2082C89
:10851000DDD3F8BD0004005070B50D4C01220421DC
:108520002046FEF7D6FB0122950329462046FEF79A
:10853000D0FB002204212046FEF7CBFB0A2002F0EC
:108540008EFB002229462046FEF7C3FB70BD0000CB
:108550000004005070B501240E4DA40300222146F2
:108560002846FEF7B6FB002204212846FEF7B1FBA1
:108570000A2002F074FB012221462846FEF7A9FBDF
:10858000012204212846FEF7A4FB0A2002F067FB23
:1085900070BD00000004005070B5144D002401228D
:1085A00004212846FEF795FB062002F058FB012225
:1085B000960331462846FEF78CFB062002F04FFB5F
:1085C00007E0641CE4B2FA2C03D9FFF7C3FF0120D3
:1085D00070BD04212846FEF76FFB0028F1D1002270
:1085E00031462846FEF775FB002070BD00040050A0
:1085F000F8B501F051FD01F081FD3B480068C0690C
:10860000FDF72EFE394D3A4E287040213046FEF7D8
:1086100053FB77010024002827D036480460A8794E
:10862000002803D10120A87102F01CF880213046F7
:10863000FEF742FB002806D0002208213046FEF754
:1086400048FB012205E0012208213046FEF741FBEC
:108650000022052039460007FEF73BFB264D274E3A
:10866000A88C274F012803D01CE0AC710022EBE757
:1086700024486946088072B680212348FDF70EFC25
:10868000002804D0022269461F48FDF7ABFC62B601
:108690001EA002F07FF8AC8403F0BAFF642002F061
:1086A000D7FAFE60688C012809D113486C844038E1
:1086B000048003F0ADFF642002F0CAFAFE60288C4B
:1086C000012806D12C8403F0A3FF642002F0C0FA35
:1086D000FE600948114A40380188914202D1C088A1
:1086E000002800D1FE60F8BDD01600203C0100201B
:1086F00000040050780100202C0E00200400FA0530
:1087000000ED00E0AAAA0000384A0008BDF8C8EB56
:10871000C9FDBCB6C4A3CABD0D0A0000AA5500001D
:1087200038B55721202000F07AF80321212000F0ED
:1087300076F84021222000F072F80821232000F072
:108740006EF8AA21302000F06AF81048018F142931
:1087500001D8002901D1012101870C4C40346188E6
:10876000142901D8002901D102216180008FC1B2F2
:10877000322000F054F8A178332000F050F8684619
:1087800000F006F80A2002F06AFA38BDEC0D00206D
:1087900010B501460F2000F021F8002800D001207C
:1087A00010BD10B50446FFF7B7FE3220FFF784FE78
:1087B000FFF7F2FEE0B2FFF77FFEFFF7EDFEFFF7F7
:1087C000ABFE3320FFF778FEFFF7E6FE0020FFF751
:1087D00043FE0446FFF7BEFE204610BD10B50C4612
:1087E000FFF7DFFF2070012010BD70B50D46044675
:1087F000FFF792FE3220FFF75FFEFFF7CDFEE0B2FB
:10880000FFF75AFEFFF7C8FE2846FFF755FEFFF7B1
:10881000C3FEFFF79FFE0A2002F021FA70BD10B5DB
:10882000FFF7E3FF012010BD10B50248FEF793FBF0
:1088300010BD000008160020FEB50446002772B6E1
:10884000334A01688B1804D13248C768032080047A
:10885000074088680190C868009048698E69002BBD
:1088600008D12C4940398B6ACD042B438B628B6A2B
:10887000AB438B62014631433CD025492368CB4250
:1088800005D12449CA6803239B049A43CA6025463C
:108890002035002810D021680A6901231A430A6193
:1088A000216848610821204600F036F8032800D1ED
:1088B000A873216808204860002E10D02068016944
:1088C000012211430161206886611021204600F0D9
:1088D00023F8032800D1A8732168102048600C48B1
:1088E0002168C14206D10B48C1680322920491431A
:1088F0003943C16020680169490849000161216864
:108900000198886021680098C86062B6FEBD0000CA
:108910000084FFBF4010024070B506460B480D466C
:10892000002409490068FCF7E3FB7D21C9004843A6
:108930003168401E00D103240B682A469A4301D0B7
:108940000028F6D1204670BD204E0000880100208E
:108950001CB5002116480091144A01910260C163C0
:108960001205426081600722826301220261024691
:10897000C16020321170FF235170C23343628162A3
:10898000117301638161042241634261C161FDF79A
:1089900081FD084800908013019069460448FDF766
:1089A00029FD00210248FDF7CFFC1CBD0024014039
:1089B000AC1500200200000408B50848016B012234
:1089C00011430163006B01211040009000220A2036
:1089D000FEF70EFC0A20FEF7FFFB08BD0010024068
:1089E000F0B587B014216846FCF7E1FB4648C26A3F
:1089F00004210A43C262C26A0A400592C16A802603
:108A00003143C162C16A31400591C16A01242143E9
:108A1000C162C16A21400591C16A02252943C16230
:108A2000C06A224628400590052010210007FEF765
:108A300050F9012235493648FEF74BF900223549F5
:108A40003348FEF746F9912105200022090200076C
:108A5000FEF73FF93048019000270520694602974C
:108A600000940007FEF76CF82C480090112001904C
:108A700003200390029769462548FEF761F810200D
:108A80006A46039591C2052069460007FEF758F82B
:108A90001120019002976946039700941C48FEF745
:108AA0004FF81F4801906946009502941848FEF758
:108AB00047F8402000906946019702951448FEF758
:108AC0003FF81848694691C1694611480397FEF777
:108AD00037F891200002694691C1052069460007D8
:108AE0000397FEF72DF8694609480197009602940E
:108AF000FEF726F8002201210520FEF779FB05206C
:108B0000FEF76AFB07B0F0BD00100240054200000E
:108B10000004005008300000000011100440000064
:108B2000000021100832000010B50F4C0D482060E5
:108B3000FF20053060600020A060E060206160617F
:108B4000E0610121206249026062A161A062072008
:108B5000E0622046FEF799FF206801684022114339
:108B6000016010BD003001403816002010B58AB0F9
:108B7000002404940594069407940894012118484D
:108B800009940094019402948907039401600921D7
:108B900084604160046113494461C160FFF740F89B
:108BA00001200003049004A90D48FFF767F80C4862
:108BB000FFF756F9089408A909480994FFF704F843
:108BC00060200090084801900294082269460394AE
:108BD0000348FFF7E1F80248FFF7B8F80AB010BD04
:108BE00090160020930400005702000000B585B0E5
:108BF00014216846FCF7DBFA0E480D490160E121BB
:108C00004902416000218160C160016181610C22E3
:108C1000C161426101623021416201210903816326
:108C20004900C163FFF750FA01F016FD05B000BD21
:108C300000380140D016002070470000F0B589B020
:108C40000A2002F057FD7D20400102F06DFDFF4C2F
:108C50000025A570FE482066607C0C2801D30B20FF
:108C6000607460790A2801D90A206071F948E570BA
:108C7000F94E00783071F949A0790978400008432D
:108C8000A17D89000843F071E06BF070010A317238
:108C9000401CE0636079B07442003046F049133004
:108CA000FCF76CFA6079EE4982004000801960316F
:108CB0001330121DFCF762FA607906214200484326
:108CC0008019E8491730921CFCF758FA2E20205ED4
:108CD000002803D0E449098A0818E0856079DB4957
:108CE000C000223182190B7B53764B7B9376062290
:108CF0007272DE4A1D301278B272A28C3273D64A7A
:108D00000B79133A1375497951750022D24902F053
:108D1000DBFD60790021C0001D3002F0E7FDD44882
:108D2000FEF7F4F901272085BF0309E0D048FEF7DC
:108D3000EDF980B22085E18EFF392D39884206DBBE
:108D400081B2E08E8142F1D3C0198142EED8022077
:108D500002F020FDC0480126C571A574A5732674D4
:108D6000E573C348FEF7D2F960850746E570607980
:108D7000FCF7E4FCBF4AC04BFCF7C4FB01F004FF66
:108D80000022BE4BFCF70CFBFCF738FD0006C00CC4
:108D9000C01980B2F103A085884201D3401AA08592
:108DA000B748E0642079401C2071B148FEF7AEF965
:108DB0002085AB48A54F643840370690B1E1AC48F8
:108DC000FEF7A4F920850BE0A948FEF79FF980B2D1
:108DD0002085A18D884203D3AA4A8918884207D3E7
:108DE00000210F2002F006FCA74920640842EBD0C6
:108DF000206C411C1FD040047ED58122D20100216D
:108E00000F2002F036FD0021102002F0F3FB410696
:108E10009348490E00227C38E16502F021FC0020D5
:108E200002F082FC002002F034FC8D487C38417A4C
:108E30000729C3D101E001F02BFD02229349401D17
:108E4000FCF7C0F90028B9D102F0A1FDE167A067E5
:108E500002F08AFD7D4B803303C3E0788049401CDB
:108E6000E07083390B7A68460370497A4170008854
:108E70000390E18C88427DD1774985488C31C98E39
:108E80000180754871498C30008F48847848FEF71E
:108E90003DF9208502F0C0FA6C48FF22803001685D
:108EA000406852040023891858410206080A1043FA
:108EB0004108490000900A0E080264498031CA60E6
:108EC00088606548E36F0A30A26F02F035FD607973
:108ED0008100614808185D49163080310CC902F0E4
:108EE0002BFD5A488030C36882685B48123002F01C
:108EF00023FD0821584800E006E14172B430C07CEF
:108F00000009607514D05648022260497738FCF792
:108F100059F900280CD15048A674C671E06D50492B
:108F20001638C2B26639C81DE274FB30FCF726F968
:108F300060790022800048491C3002F0C5FC60794D
:108F4000002180001C3002F0D1FC009802F0CBFB25
:108F5000012002F01FFC207302214E48FDF7ACFEF9
:108F600000281DD000213D4801703B498C31488EBE
:108F7000049000E05AE03881888E78818446A06CA5
:108F8000FF310531E0640860DC392065C97C0907E0
:108F9000090F032900D02175E16D1C2902D015E0CD
:108FA0000121E0E72C49294A8C31C98F1186069BA3
:108FB0002C4A1B881380884207DD002805DD002924
:108FC00003D0207E401C207600E025762571A67314
:108FD0000498B8816046F881E673608C2E49FF30B2
:108FE000C33080B2608488420CD949424018608402
:108FF00027487D220188D200491C89B20180914214
:1090000000D3058022487D210088C9004843618C37
:109010004018606500F076FD207B002805D1002116
:109020000F2002F0E7FA0006F9D583E0FCF7F6FF1F
:109030000B4A03219032115407498C314A8E3A81F0
:10904000898E7981E26D1C2A2ED127E070000020E4
:109050003F420F003C0100206012002074010020FC
:1090600090130020CC1400202C0E00204C01002076
:1090700008160020B81E85EB51B8CE3F000008400E
:10908000A0860100983A000000D027246401002047
:109090007001002000040050E7030000624B420012
:1090A000D318069A12885A808000604B5F4AD43BDE
:1090B00002905E4982189B8F138030314118A26C58
:1090C0004A605B4940185B4916300CC902F034FC19
:1090D000216EA06C884207DA544A0299515801293E
:1090E00002D12066039905915049029A895881421C
:1090F00017DD012915DD2146002812DD0398C884FB
:109100000220087065730CE04B4A00210F2002F02A
:10911000B0FB6079E178401C814202D0002002F06F
:10912000B8FA208DA18D884200D248E6434A8918BA
:109130008842FAD8A07B012801D00220A07302F057
:109140006BF93D4A00210F2002F093FB21790029A1
:1091500017D03B480288900013188B4200D225702C
:10916000002000F0E9F8A07C00283BD02F496C31AA
:109170000B78A372487860728A782272022B17D01B
:1091800030E0E16C226E323920468A420EDAC17933
:109190002B4A491CC9B2C171128852008A42E2D2DC
:1091A0000599C184022101706573DCE7E571DAE796
:1091B00010280ED0C82815D2224BC91C1D60224B86
:1091C0001818FBF7DBFF03F023FA642001F040FDE1
:1091D00031E61E4D28684000000E03D1C878FCF728
:1091E00092FA286000202378627B657910E00F4EA8
:1091F0000E4F4100303E183F765A7F5ABE4205D08E
:109200000A4F022300220126483F7E52401CC0B272
:10921000A842ECD323706273074A002180320F20EA
:1092200002F027FB09B0F0BDCC140020C0130020D1
:1092300060120020F000002000D02724983A00009F
:109240004C01002078010020EC0D00206801002076
:10925000F8B52E4C0546E06E2D4A281A411E2067AF
:10926000914215D21A21615E081AFCF753FA294A75
:10927000294BFCF747F9064632200F46205EFCF7E3
:1092800049FA32463B46FCF78BF8FCF793FA6086C6
:10929000002060761D481C23C35E828C1F48008816
:1092A00084461F4806881DE06046484380181D4FCD
:1092B00080B23880302778436427643078431A4F6F
:1092C0006066C01985420BD2C8B2184932220880A4
:1092D000606EA25E411BC9188918A166E066F8BDE0
:1092E000491C6176617EB142DED330204243104892
:1092F0006421101848430F494118E1666066322125
:10930000401B615EC0184018A066F8BD70000020C8
:10931000CF0700009A9999999999B93F5E01002069
:109320004C0100207201002078ECFFFF5C0100205E
:1093300074270000C0BDF0FFFEB5294D2988491CE7
:109340008FB228492F800E88FCF7E4F9264A274B74
:10935000FCF7D8F80191009025483146FBF7C8FE8C
:10936000244C218F4218B74206D30020288022487F
:10937000019E1018009D02E01046019E009DFCF722
:10938000DDF933462A46FCF70BF8FCF737FAA086DE
:10939000012580B2ED03A84201D3401BA086E08BDB
:1093A000FCF7CCF9154A164BFCF714F90646A08ECB
:1093B0000F460090FCF7C2F932463B46FBF7F0FF40
:1093C000FCF71CFA80B2E086A84201D3401BE0867D
:1093D0000C4900980968486100982087FEBD00008C
:1093E0005C0100204C0100201904560E2D62404003
:1093F000E17A0000700000201F050000F853E3A58B
:109400009B843E400816002070470000F0B589B0EC
:10941000002004900A2002F06DF97D20400102F046
:1094200083F9B34800228270C16BB34C491CC163FD
:10943000B049C38D098A2546C918C1852146C27520
:1094400013310791473103916D393135AB4F2230DC
:1094500005910290A64E0F21A948717100782071E4
:10946000A84AB079127840001043B27D92001043B0
:10947000E071B08FE070000A2072A17431461E22A4
:109480009C310798FBF77AFE402228469E49FBF75D
:1094900075FE029903980A7BC274497B0175092005
:1094A00060729A480078A072B08C2073F07D410001
:1094B00030469C30091805980A780275497841753C
:1094C000762000228C4902F0FFF97079062148438A
:1094D00000211C3002F00AFA022002F05BF90021A0
:1094E0000F2002F087F838423064F8D0306C411C0D
:1094F00018D040047ED58122D20100210F2002F035
:10950000B8F90021102002F075F841067A48490E9A
:109510000022B43002F0A4F87748B430417A02292E
:1095200002D0BDE001F0B4F902227949401DFBF7F9
:1095300049FE0028F5D16E480222C07D41006C48EA
:109540009C3009186C48B530FBF73CFE0028E8D188
:1095500002F01DFA664AD167906702F005FA644A84
:10956000803203C2049800282CD101200490624864
:10957000684E8C30C08E604930805D488C31098FD8
:1095800041846548FDF7C2FD5949644A0885488C05
:10959000FF30C33080B2488490420CD952428018C8
:1095A000488430885D4A401C80B20B323080904243
:1095B00001D30020308030887D22D20050434A8C75
:1095C000801848654C4869468C30428E0A80808EEF
:1095D000488049490422B531C81FFF38FBF7CEFD4A
:1095E0004348494AC07D009980001150404980316C
:1095F00003C900E075E0FF235B040022C01851415D
:109600000906060A0E43304602F06DF8710849005B
:109610000A0E0802364900268031CA608860344844
:10962000C36F826F3448483802F086F93048803082
:109630000CC83148443802F07FF92D488030C368A7
:1096400082682D48403802F077F92B4900225239C0
:109650003C2002F039F900213C2002F047F90120BA
:1096600002F098F82249087308468078401C8870F8
:1096700001210520C9030007FCF7E4FC1C48007B1E
:10968000002805D100210F2001F0B4FF0006F9D514
:10969000802200210F2002F0ECF81548467002E00D
:1096A0001349012048701248C17D491CC9B2C175D7
:1096B0000F2900D2CEE60498002810D10C4A184990
:1096C000908C002802D00B88984201D90888908499
:1096D000144980B20988401E48431349088009B0E4
:1096E000F0BD124A00210F2002F0C3F8D8E70000B5
:1096F000700000202C0E00206012002000D02724D3
:109700003C010020740100207C1400204C0100204A
:10971000640100207001002008160020E70300000B
:109720004801002046010020440100200090272429
:10973000F8B532493048086002F00EFA304800F0BF
:10974000A1F9304CE0822E48801C00F09BF9208368
:109750002B48001D00F096F960838B212A48890070
:109760004180014640310979284F0906090E617090
:1097700006D1C7800121C1870A2141870021818745
:10978000234AC18E1170C18F2171818F6171817ADD
:10979000A17085880521A5626181C6883046FBF7E6
:1097A000A7FCA08101462846FBF7A2FC8800081808
:1097B00085B2164825816843FBF7C0FF154A164B52
:1097C000FBF708FFFCF71AF8E0816582314638465E
:1097D000FBF78EFC20820146C820FBF789FC6084E1
:1097E00001202084FCF732FCA082E2890B490C485E
:1097F000FDF790FCF8BD000085A600086800002079
:10980000004F00083C010020EC0D0020E8030000A0
:1098100018000020F853E3A59B843E40FF7F000022
:1098200008160020F8B5744C00202071734D0120FB
:109830002880734EC8203080E07A401CE072C00758
:1098400006D0A08C411EA184022801D2C820A08489
:109850000120C043FFF770FD0A2001F04BFF7D207F
:10986000400101F061FF02216648FDF725FA00285A
:109870007ED00020644980000978654F4900084384
:10988000624909780843B872102078726148C1882B
:109890007D20C000FBF72CFC78735F485D490078A1
:1098A000B87338460B308A780270C97841705949CC
:1098B000421C20310B7ED370497E11715549D01C5A
:1098C00022310B7E5371497E9171524940310A7C9D
:1098D0000271497C417100223946172001F0F4FFE2
:1098E0000021172002F002F8022001F053FF4B4F35
:1098F00000210F2001F07EFE38422064F8D0206C59
:10990000411C77D0400471D58122D20100210F2063
:1099100001F0AFFF0021102001F06CFE41063C4831
:10992000490E0022B430E16501F09AFE384FB43799
:10993000787A11285AD102223949781DFBF742FC66
:10994000002853D1F81F027A69460A70407A48709D
:10995000B97A2980C820FBF7CBFB3080387BA08404
:109960003846304D2838C08E28802348394600E0DC
:109970003EE02839098F41842B48FDF7C7FB20853D
:10998000608C2A49FF30C33080B2608488420CD991
:1099900049424018608428882449401C80B20B3119
:1099A0002880884201D30020288028887D21C90092
:1099B0004843618C4018606500F0A4F86846008850
:1099C000E0841349B87CC7316071420008460D46F7
:1099D0006930FBF7D3FB6079294642001448FBF756
:1099E000CDFBA08CFF2801D003202070F8BD01E042
:1099F00001203FE700F04CFF700000204C010020E8
:109A00005E010020000400504001002041010020C0
:109A100060120020EC0D00201800002000D0272448
:109A2000640100207001002008160020E7030000F8
:109A3000A813002070B586B014216846FBF7B7FB69
:109A400001250F4EED03002229463046FDF741F96E
:109A50000120002401900294694600950394304649
:109A6000FDF76EF803200190029469460095039477
:109A70003046FDF765F8022001F0EAF806B070BD47
:109A8000000400500088704770470000F8B5044695
:109A900000206A461080194D55222A70AA226A7049
:109AA0000322AA70661DEE702A716971144A49007A
:109AB0008918AC712246E81DFBF760FB002007E027
:109AC00029186A468978128889186A461180401CCC
:109AD000B042F5DB611DA81CFCF716F9014668468B
:109AE000018029190078C8716846407808722146BB
:109AF0000931024800F0DCFBF8BD000046150020EB
:109B0000EC0D0020FEB5FFF7A3FB2548FDF7FEFA9C
:109B1000244C86B2268560790A21081AC000FBF71A
:109B2000F9FD07460191A06EFBF708FE1E4A1F4B88
:109B3000FBF750FD00900D463046FBF7FFFD2B462E
:109B4000009AFBF72DFC3A46019BFBF729FCFBF73B
:109B500055FE85B2A586E08BFBF7F0FD124A134B4C
:109B6000FBF738FD06460F462846FBF7E7FD324671
:109B70003B46FBF715FCFBF741FE81B20120C00319
:109B8000E186814201D3091AE186854201D3281A70
:109B9000A0860349A08E096848612087FEBD0000A9
:109BA0000816002070000020F853E3A59B843E4077
:109BB000034A1168382389B2994301431160704701
:109BC0000030014010B5FDF791F810BD10B59AB006
:109BD00034216846FBF7EBFA14210DA8FBF7E7FAEE
:109BE0001C2112A8FBF7E3FA1B4801680324E402D6
:109BF000A143C21489180160FDF706FB17480169EB
:109C0000A143016106200090FF2001300290012055
:109C10000390102004900220099040040B90000152
:109C200000240C900A946846FDF71CFD0F200D904F
:109C300003200E900F941094012111940DA8FDF7AC
:109C4000E7FB81201290032080041890149412A83E
:109C5000FDF72CFB1AB010BD007000404010024010
:109C600010480168821511430160C1680E4A114015
:109C7000C16001680D4A11400160816849084900CE
:109C8000816001680122920491430160C168FD2254
:109C900012049143C16000210161064904488860B3
:109CA00070470000001002400C40FF88F6FFF6FEEF
:109CB0000050000800ED00E070B5026801239B072A
:109CC000114C124D984203D0A04201D0A84203D1BA
:109CD0007026B2434E683243984203D0A04201D06E
:109CE000A84204D103231B029A43CB681A43802362
:109CF0009A430B691A4302608A68C26209688162EA
:109D00000121416170BD00000008014000140140C4
:109D100030B58468FF252D021B021343AC430B436F
:109D20002343836030BD826870239A430A4307212E
:109D30000A438260704730B5026A520852000262DC
:109D4000026A456883697024A3439C080B68A400D9
:109D500023430224A2438C6845601443836149680D
:109D60004163046230BD30B5026A10239A43026237
:109D7000036A4568826973242402A2430C682402A2
:109D80001443202293438A68456012011A43846178
:109D900049688163026230BD30B5026AFF23013336
:109DA0009A430262026A4568C3697024A3439C080F
:109DB0000B68A400234301246402A2438C6845601D
:109DC00024021443C3614968C163046230BD30B5E5
:109DD000026A01231B039A430262036A4568C2694F
:109DE00073242402A2430C68240214430122520368
:109DF00093438A68456012031A43C4614968016449
:109E0000026230BD30B5036A046A6408640004620B
:109E10008469F025AC43120122430A24A3430B4377
:109E20008261036230BD30B5036A1024A34303622C
:109E30008469036A0F252D031203AC432243A02437
:109E4000A343090119438261016230BDF8B51024B2
:109E500005252D07AC62AF20800000F000FFAC614B
:109E600001F0DCFB344C354F354E60670EE001F0FD
:109E7000D5FB6067FEF7BCFB606C411C6164142875
:109E800004D930A000F086FC3248C760606FB04251
:109E9000EDD10026666420780127FF03030000F05F
:109EA000B2FC05040C192D3A3C0001223946284623
:109EB000FCF70FFFFFF7B6FC06E001223946284603
:109EC000FCF707FFFFF7A2FA002239462846FCF705
:109ED00000FF22E0607B0122401C60733946284667
:109EE000FCF7F7FEFCF7CEF8002239462846FCF7CF
:109EF000F0FE607B052810D926700EE0FEF79EFE6E
:109F0000FCF762F9154814490068FBF7C1F9FBF743
:109F100023FCE08501E0FFF779FA02211048FCF705
:109F2000CBFE002805D000200E49087001F05CFA35
:109F3000F8BD0120F8E70000700000200400FA05D9
:109F40003001CADE4457204944204552524F522E18
:109F50000D0A000000ED00E00000C84200000020F3
:109F6000000400507401002010B5818CC90707D08F
:109F700001684A6801235B049A43836A1A434A6072
:109F8000818C890707D501684A6801231B049A431D
:109F9000C36A1A434A60818C490707D501684A6839
:109FA00001239B049A43036B1A434A60818C09077F
:109FB00007D501684A680123DB039A43436B1A43C0
:109FC0004A60818CC90607D50268916801231B038A
:109FD0009943836B19439160818C890607D5016889
:109FE0008A6801235B039A43C36B1A438A60818C9E
:109FF000490612D503685A6801210905046C8A4391
:10A0000022435A60026C8A4207D1026851680323D6
:10A010005B059943436C19435160818C090607D550
:10A0200001684A680123DB04806C9A4302434A605A
:10A0300010BD0000F8B50446002680300660FCF72D
:10A040004FFE054620680068124F000709D5012120
:10A050002B46002249052046009700F0A1FA00286F
:10A060000DD12068006840070BD501212B46002246
:10A0700089052046009700F093FA002801D00320BC
:10A08000F8BD2020A067E0672666603426750020B2
:10A09000F8BD0000FFFFFF01F8B5154CC826E078B9
:10A0A000002823D16079002820D101206071114D52
:10A0B000686B0027002818D0686BC821081A0FE0C9
:10A0C0000D48E168405C61698847E068401CE060D9
:10A0D000E068C82800DBE760696BC820401A761E7C
:10A0E000E168814201D0002EEADC6771F8BD000012
:10A0F0005400002000000240240D002070B5224CC6
:10A10000E07800283FD1207900283CD1012020713F
:10A110001E4EF16900250906002933DA21566257DF
:10A1200091420AD1F06940062CD5A079002829D0A7
:10A13000A5712089401C208124E0A179002903D148
:10A14000A0710A2000F08BFD00202056CC2148434E
:10A150000F494218206912181279B262401C00227D
:10A160002061A256CC235A43895881420ADC2561DA
:10A170002078401C207020780E2800D12570A0780F
:10A18000401CA070257170BD5400002000380140B3
:10A19000FC01002010B5806A0022014640314A834C
:10A1A0004A82FDF77FFE10BD70B5846AA06FE56F2F
:10A1B0002168896800260906002906DA212804D1C9
:10A1C00052200653204600F06BF820688068400655
:10A1D00006D5222D04D15A200653204600F047F818
:10A1E0002046803001681022114301602046FDF7AF
:10A1F00059FE70BD10B501460968806A0968890674
:10A200001CD400225A210A5201680A68FF23013334
:10A210009A430A6001688A68520852008A6001689D
:10A220008A6840239A438A602021C167016E012910
:10A2300004D101680A6810239A430A60016E01295B
:10A2400002D0FEF711F810BD5821095AFDF728FE7B
:10A2500010BD10B5806A016E012902D0FEF705F825
:10A2600010BD5821095A4908FDF71AFE10BD0168B2
:10A270000A68FF2321339A430A6001688A685208FA
:10A2800052008A60016E012904D101680A68102316
:10A290009A430A602021C167002101664166704728
:10A2A00001680A68C0239A430A60202181677047C9
:10A2B00070B5164CE278002A0CD12279002A09D117
:10A2C0000122E2700025C82903DC0222A256002ADE
:10A2D00001DCE57070BD0123E356CC2253430C4AE8
:10A2E000D1500123E356CC2673439B180A460146FE
:10A2F000181DFAF743FF6078401C607060780E28E4
:10A3000000D16570A078401EA070E2E754000020E4
:10A31000FC010020F8B50446016880682369E669FD
:10A3200018436369002533431843724A0B68724E21
:10A33000334003430B602168486803231B039843A1
:10A34000E368184348602168A069914201D0236AFC
:10A3500018438B680B263602B34303438B6067496F
:10A36000236867488B420CD1C0688007800F06D0F5
:10A37000012839D0022835D0032821D11EE0012739
:10A380001FE060498B420AD1C0680C21084027D0E9
:10A39000042829D0082825D00C2811D10EE093429A
:10A3A0000ED1C16803208002014019D00120800233
:10A3B000091A19D0091A15D0814201D1082700E0E5
:10A3C00010274F49504840398600934232D1002F20
:10A3D0000CD0022F0DD0042F10D0082F7FD126E0F3
:10A3E0000027EEE70227ECE70427EAE7FDF7DEF8AF
:10A3F00006E00968C90605D4304603E0FDF7F6F823
:10A40000002872D0626851005118814267D8110348
:10A41000814264D3010E06025008002330185941CE
:10A42000FAF77CFE03210902411A384A55E001205F
:10A43000C003E7E70122E369D20393422BD13B003B
:10A4400000F0E1F90906090C4D114D4D4D274D0065
:10A45000FDF7ACF809E0FDF7B9F806E00968C906B0
:10A4600005D4304603E0FDF7C1F800283DD061680F
:10A4700040004A088018FAF73BFE80B20146244AA1
:10A48000103991422BD8511C01400007400F08435E
:10A4900029E01046EBE73B0000F0B5F90906090C8E
:10A4A0002112212121232100FDF780F80AE0FDF788
:10A4B0008DF807E00968C90606D4304604E00EE0CE
:10A4C000FDF794F8002810D061684A081018FAF7D0
:10A4D0000FFE80B201460E4A1039914203D9012580
:10A4E00003E01046F0E72168C86000206066A066BF
:10A4F0002846F8BD00480040F369FFEF00380140EE
:10A50000401002400044004000093D00FFFC0F00E5
:10A51000EFFF0000F8B504464165403000262746AD
:10A52000028380373E602220E0672546206F603539
:10A5300000281CD01749C162216F17480863216F9A
:10A5400016484863206F8663236F606D9C461346F0
:10A550002168024660462431FCF71AFA002806D02A
:10A56000102038602E752020A0670120F8BD2E75C0
:10A5700020680168FF220132114301602068816870
:10A58000012211438160206881684022114381606B
:10A590000020F8BDF5A1000853A20008A9A10008F9
:10A5A000FFB581B005460F46044660350A9E39E086
:10A5B000701C37D0FCF794FB0499401AB04222D8A3
:10A5C000002E20D02068016849072BD5C069C04300
:10A5D000000527D401202168C002086220680168B4
:10A5E000FF22A13291430160206881684908490037
:10A5F00081602020A067E0678034206000202875FB
:10A60000032005B0F0BD20680168FF22A13291430C
:10A610000160206881684908490081602020A067A6
:10A62000E067EBE72068C1693846884305D0002120
:10A6300003988142BCD00020E3E70121F8E7000045
:10A6400010B504491020096808620248FDF72CFC87
:10A6500010BD0000D016002001490D208870704701
:10A660005400002010B5FEF7A7F9FEF7BFFAC82284
:10A6700002490348FDF7C8FD10BD0000240D00206D
:10A68000D0160020F8B53E4C002321783D4A1D46E7
:10A69000082910D0072947D0062950D0052952D0C3
:10A6A000042953D0032954D0002956D0012958D069
:10A6B00002295AD05BE0A17800264A1F04E0314FFE
:10A6C000BF5DFB189BB2761C9642F8DB6679277952
:10A6D0009A195118E3786278C9188918C91940186D
:10A6E000C0430006000E1AD1012E14D0022E16D13E
:10A6F00025482449C018FAF741FD01F089FF64207C
:10A7000000F0A6FABFF34F8F21492048C860BFF37D
:10A710004F8F00BFFDE759081046FFF7B7F92570C6
:10A72000E570A570A571F8BDA1795054491CC8B257
:10A73000A071A178491F8842F5D1082001E060701E
:10A7400007202070F8BDE0700620FAE76071052050
:10A75000F7E7A070E5700420F3E7552807D1012042
:10A76000EFE7AA2803D10220EBE7032803D02570E6
:10A77000E570A570F8BD032020702071F8BD0000C1
:10A7800034010020E2140020EC0D00200400FA0542
:10A7900000ED00E010B5024A024900F0E5F910BDF5
:10A7A00051B900088C0100202021020C01D0102199
:10A7B0001046020A01D010460839020901D010469D
:10A7C000091F820801D01046891E420801D0881E48
:10A7D0007047081A7047F8B5040C8BB2264682B24F
:10A7E0005E430D0C1046370C584336048019002187
:10A7F000794116466E43370C360480197941264656
:10A800006E438919F8BD30B47446641E2578641C03
:10A81000AB4200D21D46635D5B00E31830BC1847B5
:10A820004900CA020243100000D004204A0D01D0A2
:10A8300001221043044A490D914201D102210843EB
:10A84000012800D105207047FF0700008307FF2281
:10A85000DB0E9A408907090E9940002808DB83081F
:10A8600009489B001B1818689043084318607047FC
:10A870000007000F0838830804489B001B18D8699C
:10A8800090430843D861704700E400E000ED00E029
:10A89000BFF34F8F04490348C860BFF34F8F00BF19
:10A8A000FDE700000400FA0500ED00E0F8B50446FD
:10A8B0004F1EC8000838211815461E46086849680A
:10A8C0003A4606239A4310D02A463346FAF71AFE30
:10A8D0003A46D200083AA3181A687F1E5B68FAF756
:10A8E0005FFD06223B469343EED1022F23D0042F77
:10A8F00011D0062F2FD12A463346FAF703FEE36A1A
:10A90000A26AFAF74DFD2A463346FAF7FBFD636A61
:10A91000226AFAF745FD2A463346FAF7F3FDE36962
:10A92000A269FAF73DFD2A463346FAF7EBFD636963
:10A930002269FAF735FD2A463346FAF7E3FDE36864
:10A94000A268FAF72DFD2A463346FAF7DBFD636865
:10A950002268FAF725FDF8BD002210B5134610460F
:10A960000149FAF737FE10BD0000F03F10B5FAF7C5
:10A9700017FD10BD002210B5134610461146FAF718
:10A9800029FE10BD10B50721024A00200907FAF779
:10A9900099FE10BD01030000034A10B50020110705
:10A9A000FAF790FE10BD000001FDFFFF02E008C8AD
:10A9B000121F08C1002AFAD170477047002001E039
:10A9C00001C1121F002AFBD1704700000149086035
:10A9D000704700009001002008B500216846017012
:10A9E0006B46012202212C2000F052FF0221684612
:10A9F00001706B4601222C2000F04AFF08BD0000C8
:10AA000038B504466D20694608706B460122074937
:10AA10002E2000F03DFF0649002C01D0054A00E041
:10AA2000054A2E2000F01AFF38BD0000060800007D
:10AA300006180000070600000716000038B5044697
:10AA40006B4602220021362000F0EEFDB3212300E8
:10AA5000FFF7D9FE0E0F08153A3A3A3A1C273A3A50
:10AA60002F34483A00216846017040784108490077
:10AA700014E06946087880088000401C04E06946BC
:10AA8000087880088000801C08701DE06846027805
:10AA90000A40483202704178802001436846417084
:10AAA00012E0684602780A40027040784106490E7A
:10AAB000F4E7694648780221084303E0694648788C
:10AAC000FD210840694648706B460122002136206E
:10AAD00000F0DEFE012200AB11463620013300F00B
:10AAE000D7FE38BD69460878CF2108406946203036
:10AAF000CAE708B5032168464170012101706B4621
:10AB000002220021362000F0C3FE0122D2030621DA
:10AB10002D2000F0A3FE012000F09AF80120FFF79D
:10AB20008DFF08BD08B5020A69464A7008706B4679
:10AB3000022204212D2000F0ABFE0320694608709C
:10AB40006B46012206212D2000F0A2FE002069465E
:10AB500008706B46012206212D2000F099FE0A2183
:10AB60002D2000F047FD08BDF8B516460F460446F7
:10AB7000002503E03946B047641C6D1C207800288E
:10AB8000F8D12846F8BD0000F8B54A002B4B520D0D
:10AB9000D6182B4A0C460546142E2BDA002E12DA54
:10ABA000284BFAF7FDFB00221346FAF76DFE40D260
:10ABB000002C03DA0124E40700253AE0204628436C
:10ABC00037D0214C14E0214F0B46F7403B402B433C
:10ABD00031D01C4BFAF7E4FB00221346FAF754FE7F
:10ABE00027D2002C03DD01200005F0400419BC43EE
:10ABF00000251EE0332E1EDC33460027143BFF43A6
:10AC0000DF40384217D00F4BFAF774FC002213468E
:10AC1000FAF73AFE0DD2002C0ADD142E0CD03420A7
:10AC2000811B012088404019A84200D2641C0546BF
:10AC3000BD4321462846F8BD641CF9E701FCFFFF2F
:10AC40009C7500883CE4377E0000F03FFFFF0F005A
:10AC50007D2110B5C900484300F001F810BD002166
:10AC600040E000BF00BF00BF00BF00BF00BF00BF8B
:10AC700000BF00BF00BF00BF00BF00BF00BF00BFDC
:10AC800000BF00BF00BF00BF00BF00BF00BF00BFCC
:10AC900000BF00BF00BF00BF00BF00BF00BF00BFBC
:10ACA00000BF00BF00BF00BF00BF00BF00BF00BFAC
:10ACB00000BF00BF00BF00BF00BF00BF00BF00BF9C
:10ACC00000BF00BF00BF00BF00BF00BF00BF00BF8C
:10ACD00000BF00BF00BF00BF00BF00BF00BF00BF7C
:10ACE00000BF491C8142BCD37047FFB581B01E46EE
:10ACF0000F46040026D00B9903980143A06A3943FC
:10AD0000826807209047002818DB0A99A06A31431F
:10AD1000826806209047002810DB25462035A97957
:10AD2000032F01D908200143032E01D90420014338
:10AD3000A06A826809209047002806DA0120C043F3
:10AD400005B0F0BD0020C043FAE7384600F000F936
:10AD50002060304600F0FCF860600A986870039844
:10AD6000A870EF702E710B9868710020E8E7000062
:10AD7000F7B50446002090B000900190002C05D05B
:10AD80006A46062101F07EFC062803DA0020C04353
:10AD900013B0F0BD684640780102684600780004B0
:10ADA0000918684680780818FAF7C8FC054668460E
:10ADB0000391007901026846C078000409186846CA
:10ADC00040790818FAF7BAFC032206460F469207A4
:10ADD0005C4BFAF759FD07D200225B4B30463946EF
:10ADE000FAF782FB06460F4603229207554B284688
:10ADF0000399FAF749FD07D20022534B28460399DD
:10AE0000FAF772FB054603912068FAF797FC0246B1
:10AE10000B4630463946FAF7DDFB07460A20079114
:10AE2000205EFAF777FC3A46079BFAF76BFB06467B
:10AE300008200991205EFAF75BFC0021C943FAF76C
:10AE4000A2FAFAF7F9FC3246099BFAF7A9FA069139
:10AE500008906068FAF772FC02460B462846039990
:10AE6000FAF7B8FB05461A200E46205EFAF752FCA8
:10AE70002A463346FAF746FB0C9009911620205ECD
:10AE8000FAF748FC099B0C9AFAF78AFA05910A909E
:10AE90002A46334638460799FAF734FB059B0A9A47
:10AEA000FAF730FB05910A901420205EFAF732FC85
:10AEB0003A46079BFAF726FB07461C200791205EBF
:10AEC000FAF728FC2A463346FAF71CFB0E900B9142
:10AED0001820205EFAF71EFC0B9B0E9AFAF760FA18
:10AEE0002A463346FAF70EFB0B910E902069FAF7CB
:10AEF00011FC0B9B0E9AFAF753FA2A463346FAF7DF
:10AF000001FB05460E46E068FAF704FC2A46334684
:10AF1000FAF746FA3A46079BFAF742FA059B0A9A6D
:10AF2000FAF73EFA01229207084BFAF7EBFA0246CB
:10AF30000B46129C0898069903C411980CC0002077
:10AF400026E70000FFFF5F4100007041E17A843F87
:10AF500000B50121C9040300FFF755FC081A0508D4
:10AF60000B0E1114171A0320C00400BD0720C004E3
:10AF700000BD0F20C00400BD1F20400300BD3F20C6
:10AF8000400300BD7F20400300BDFF20400300BD03
:10AF9000084600BDFEB5264F0D4604000FD0002D1B
:10AFA0000DD0264600202036B071F07129680D20A2
:10AFB0008847002801DA7800FEBD102801D0384605
:10AFC000FEBDA562E968002901D0282088472046F7
:10AFD00000F030F80028F3DBA06AA52182680E207B
:10AFE0009047A06A962182680F209047A06A0221AC
:10AFF000826862209047A06A002182680E209047F4
:10B00000A06A002182680F20904771793020019159
:10B0100000900623202201212046FFF766FE00282B
:10B02000CEDB204600F0AEF80028C9DB0020FEBDD4
:10B03000FFFFFFFF10B586B0044614216846FAF7FB
:10B04000B6F8002C7ED0A06A122143686A46102010
:10B050009847122877D16846007801220101684696
:10B06000407812030009081843492081884201DD15
:10B07000801A20816846837840780007000D1818F0
:10B080006081884201DD801A608168460079012272
:10B0900001016846C0781205000309186846407926
:10B0A000000908183549E060884201DD801AE06037
:10B0B000684640790007030B6846807900021B1838
:10B0C0006846C07918182061884201DD801A206125
:10B0D0006846417A007A0002081802B22848012125
:10B0E0000904A282824201DD521AA2826A46D37A00
:10B0F000927A12029A1812B2E282824201DD521A48
:10B10000E2826A46537B127B12029A1812B22283A1
:10B11000824201DD521A22836A46D37B927B12025D
:10B120009A1812B26283824201DD521A62836A4621
:10B13000537C127C12029A1812B2A283824204DD5E
:10B14000501A01E00BE008E0A083A06A0168282003
:10B150008847002806DA0120C04306B010BD002051
:10B16000C043FAE7C011C0072034002800D0802077
:10B1700060710020F1E70000FF070000FFFF0700FB
:10B18000FF7F000010B5040009D0A06A0721826883
:10B1900008209047002805DA0120C04310BD002098
:10B1A000C04310BD072020342070002010BD0000D7
:10B1B000FEB504460020019000906079734940007C
:10B1C0000E5A61782578491E7148CFB20163042D6B
:10B1D00077D0072D75D000210291217801736C4939
:10B1E000E379012292058969002B6CD0914381613A
:10B1F0006748217A4173217A82698907890B0A435A
:10B2000082610021042000F034FB324661492E2087
:10B2100000F024FB3846FFF7F3FB5F4E0522705D1C
:10B22000810040185D49431807212B2000F030FBB6
:10B230005B49029801220B180B21282000F028FB03
:10B24000705D584980000A580C21282000F011FB3D
:10B25000E079554980004018A1794900425A0221FD
:10B26000272000F0FBFA51487E00825B0421272052
:10B2700000F0F4FAE079002829D0A07804282CD036
:10B2800028206946087220220621272000F0E6FACD
:10B2900002AB01222621272000F0FAFA44493801A6
:10B2A0004018E178890042580821272000F0E1FA8F
:10B2B000A17A601C627A0902114313D016E000E003
:10B2C00001E0012188E71143F608816190E76422DB
:10B2D0000621272000F0C2FAE0E710206946087234
:10B2E0000246D1E733490172090A4172417A007A74
:10B2F0000A0202432021272000F0B0FA2E4F0C2131
:10B3000023203A6800F0B5FAF0198288042123203E
:10B3100000F0A4FAA07900280BD0E0792749012297
:10B3200043180021212000F0B3FA032001900120EE
:10B3300000902A07120F1001024360780021800755
:10B34000000B0243019800050243009840040243A9
:10B350002079C006400902436079C00602431F20DD
:10B3600000F087FAA07861780123084302040848B6
:10B37000DB030261E179490319430A4302610021B9
:10B38000082000F076FA0020FEBD0000B8C70008D3
:10B39000C00100200428000060C70008240000202D
:10B3A0004200002068C7000888C7000894C700084A
:10B3B00098C700084110000080C700084400002022
:10B3C00038B50C4607498A8B002102432C2000F037
:10B3D00045FA684604706B46012206212C2000F0D5
:10B3E00057FA38BDC001002010B5FFF7F5FA10BDBF
:10B3F00010B504460421362000F0FCF80121C902F2
:10B40000002C01D0084300E0884302460421362086
:10B4100000F02FFA10BD000038B5402069460870D2
:10B4200000210E2000F0E6F80446002211460E200E
:10B4300000F01FFA6B46012200210D2000F028FACF
:10B44000074A00210F2000F014FA00F0EDF922461F
:10B4500000210E2000F00DFA02480021017338BDD2
:10B46000F8FF2724E0010020FEB5054604206946C8
:10B470000870514C002060752146203120634871CE
:10B480000873A0836063A06300F0C8F84B4E20608F
:10B4900002E000F0C3F82060B042FAD10020FFF7CC
:10B4A000CDFA00F0BBF8464E20603078242801D950
:10B4B000243806E00621F9F71BFE0622101A400187
:10B4C0000843020601040A4301020A430243B26030
:10B4D000706000211E2000F0CCF900F09FF8206081
:10B4E0006B4601220021242000F0D2F91E20FFF734
:10B4F00019FB86B2300AA0730420FFF713FB07463E
:10B5000000F08CF820603806000E0DD0022069464D
:10B51000087101AB012212212D2000F0B9F9A08B96
:10B52000012109030843A08300F078F82060062079
:10B53000FFF7F8FA60600720FFF7F4FAA060F00662
:10B54000C00E207501D110202075C0B200F0DCF9CA
:10B55000E80707D0FFF7CDFAA08B0121C902084305
:10B56000A0830AE00521362000F02EF81549084096
:10B5700002460521362000F071F90120FFF75EFA3E
:10B580000021042000F036F8A0610021262000F000
:10B5900031F815218903084302460021262000F0D6
:10B5A00068F900222621362000F058F900F036F81C
:10B5B00020600020FEBD0000C00100203001CADE76
:10B5C00018000020FFFD000038B5094C89B280B298
:10B5D0006B46022200F028F8002806D16846407821
:10B5E000010268460078081884B2204638BD000081
:10B5F000FFFF000038B50024E44389B280B26B46F7
:10B60000042200F011F8002806D103216846435CAB
:10B610002202D418491EFAD5204638BD10B50021A3
:10B620000846FFF7E7FF10BD38B5002909D04024D0
:10B6300020436C462070C8B27F2906D86070022073
:10B640000AE069460870012006E0802420436C4629
:10B650006070C809A0700320694600F0B3FF38BDD0
:10B6600010B5144603460A4621461120FFF7DCFFB9
:10B6700010BD10B50346052200211520FFF7D4FFA9
:10B6800010BD10B50346052200211720FFF7CCFF9F
:10B6900010BD38B5054600206946087000F0C4F8B2
:10B6A000FF2401342246002D01D003221202002182
:10B6B0000D2000F0D3F8002D13D06B46012203219A
:10B6C0000F20FFF7B1FF68460078000709D5FFF7A4
:10B6D000A3FE224600210D2000F0C0F80020C04348
:10B6E00038BD002038BD10B5024601210A2000F007
:10B6F000C0F810BD10B5044600211A20FFF77AFFEC
:10B70000000D22030005120B024300211A2000F055
:10B71000B0F810BD10B5024602492E2000F09EF888
:10B7200010BD000004180000F8B505466B46012264
:10B7300003210420FFF778FF0126114C3607002D66
:10B740000DD02A4600210C2000F088F869460878C0
:10B750001021084369460870A069304307E0694634
:10B760000878EF21084069460870A069B0430B468D
:10B77000A06101220321042000F08AF8F8BD000036
:10B78000C001002010B502460021182000F066F824
:10B7900010BD0000F8B50746002568460570B807DB
:10B7A000204C2E4600280ADA8020694608706B4635
:10B7B000012200210D2000F06BF801202073F80712
:10B7C0006946087821D006210843694608706B460F
:10B7D000012200210D2000F05BF803210F20FFF76C
:10B7E000F3FE8121C900084219D040206946087043
:10B7F0006B46012200210D2000F04AF80020FFF7DF
:10B80000F7FD00252673ED4309E002210843694650
:10B8100008706B46012200210D2000F039F82846FF
:10B82000F8BD0000E00100201CB56B460122032199
:10B830000F20FFF7F9FE684600784022C10910404A
:10B84000C9014000814208D00120694608710246C2
:10B8500001AB03210D2000F01BF81CBD08B56B46A1
:10B860001A70120A5A7089B280B2022200F010F8DF
:10B8700008BD38B500236C46E254120A5B1C042B49
:10B88000FADB89B280B22346042200F001F838BD09
:10B8900038B58024002909D0C02528436D4628707A
:10B8A000C8B27F2907D86870022009E020436946A2
:10B8B0000870012004E020436870C809A8700320C4
:10B8C000694600F029FF38BD10B51446012312184F
:10B8D0009B029A4202D90020C04310BD0B46821E33
:10B8E00021460920FFF7D4FF002010BD10B5054AFE
:10B8F0008905126901430A4300210820FFF7B9FFB7
:10B90000002010BDC001002038B504466B4601225E
:10B910000E212B20FFF788FE68460078E1064009DB
:10B920004001C90E0143684601706B4601220E2199
:10B930002B20FFF7ADFF38BD10B5002142541C0687
:10B94000120A22431B0A491C0429F7DB10BD000020
:10B9500013B501231A4669460248FCF787FC009894
:10B960001CBD0000D01600207CB50024254668468A
:10B97000FFF77FFE04206946220E2D0215432202A6
:10B980000C5C1443401EF7D5204629467CBD7CB58F
:10B99000002425466846FFF774FE04206946220EFF
:10B9A0002D02154322020C5C1443401EF7D520469D
:10B9B00029467CBDFBF7A2F9FEF708F9FDF710F860
:10B9C0003F494048002522C005608561C5613E4968
:10B9D0000562C1600838FBF723FBFCF7EDFFFDF7BC
:10B9E00005F9FDF7A1F8FCF7B3FF052401222407B0
:10B9F000D1032046FBF76DF9FDF79AFEFCF790FEA8
:10BA0000FAF724F9FAF7E0F9FAF7AEF9FCF7B0FC27
:10BA10000721A015FFF7D4FCFFF7E6FC0122110374
:10BA20002046FBF756F92748C8222849C830FCF7BA
:10BA3000EBFB274F274E284C387800280ED1307862
:10BA4000002801D0032809D140212448FBF734F90C
:10BA5000002803D101210846FBF7F6FBE078002817
:10BA60002AD06078002827D0E57072B620780F2899
:10BA70000AD90120194900038861FEF7E7F901207E
:10BA80001649000388620CE0012251031348FBF7BA
:10BA900020F9FEF7DBF90121002249030F48FBF7EB
:10BAA00018F962B6FCF7A4FDFAF7F4F8A08C0028A8
:10BAB000C2D0401EA084BFE7FCF79AFDBCE700009F
:10BAC000007C004008160020FFFF0000240D00202D
:10BAD0005A000020840000203C0100200004005097
:10BAE00010B586B01748FBF71EFA14216846F9F71F
:10BAF0005EFB154800900320019000200290052075
:10BB000069460007FBF71CF869461048FBF718F870
:10BB100069460F48FBF714F801210846FBF794FB30
:10BB2000FF2401342046FBF767FB0A49086804221A
:10BB3000104308602046FBF76FFBFBF775FB06B070
:10BB400010BD000008160020FFFF00000004005098
:10BB5000000800500070004010B501229202164902
:10BB60001648FAF7B5F91448154902888A4222D0D6
:10BB7000018014498180FF21F531C1800A210181B2
:10BB800000211E224181D24382810122C281818310
:10BB90004323C3860287782343878287C28702466E
:10BBA0004032118451849184C18391801423838213
:10BBB000118200F02DFD10BDEC0D002000FC0008EE
:10BBC000AA55000034120000F0B51FB496B08446A8
:10BBD0000C460246199D18980390490068006300BE
:10BBE000490840080193002A01D0012600E0002600
:10BBF0009E19FE4BF6185B109E422BD36E00039FDE
:10BC00000296002F00D00127F719F84EF84BBE1905
:10BC10009E421FD3039E0346F64F334309D03B4653
:10BC20009C4201D1002A04D0019B002A05D00126A4
:10BC300004E0002039461BB0F0BD00269E19EE4BF3
:10BC40009E4207D8039F029E002F00D00127F619BD
:10BC50009E4207D92B4660462146189AFEF786FE7B
:10BC60001BB0F0BD0023002C29DAE44EB04226DAE6
:10BC7000E34EB04201DB022321E0DE4EB0421EDB88
:10BC8000E04E070DBE19142E09DD3427BF1B039E9D
:10BC9000FE400196BE40039FBE420BD00FE0039FC3
:10BCA000002F0CD11427BF1B0646FE400196BE4054
:10BCB000864204D1019BDE07F60F02239B1B0E4632
:10BCC000164318D1002D16DA002C03D0022B01D018
:10BCD000012B06D00220FEF779FEFEF73DFE1BB0D9
:10BCE000F0BD0220FEF772FEFEF736FE0122D207FB
:10BCF00051401BB0F0BD039E002E61D1BF4EB0423B
:10BD000020D1C148844201D1002A08D0B9488142DB
:10BD100009DB002D10DB189829461BB0F0BD002070
:10BD2000B4491BB0F0BD002D06DA01222946D20726
:10BD3000189851401BB0F0BDB4497944086849686F
:10BD40001BB0F0BDAB4FB84225D1002D1FDA002942
:10BD500004D0B14212D1002A09D018E0002A72D1D1
:10BD6000A649E20F0020D20711431BB0F0BD00200E
:10BD7000E20F0146D20711431BB0F0BDB14206DA13
:10BD8000234600203946F9F725FC1BB0F0BD1046CC
:10BD900021461BB0F0BDB14212DA0126B607B5420A
:10BDA00003D1234610461946FEE3994EB54207D10A
:10BDB000261E05DB1046314600F040FC1BB0F0BDEE
:10BDC00067007F081646002A40D100290AD08B4A16
:10BDD000914229D1002C0EDD002D1CDB00201146E4
:10BDE0001BB0F0BD022B16D0002C14D0012B12D1A9
:10BDF000002C14DB0FE0002C28DA002D09DB012BCE
:10BE000003D000207D491BB0F0BD002081491BB04C
:10BE1000F0BD012B03D0002001461BB0F0BD002077
:10BE20000121C9071BB0F0BD724A91420ED1002C0E
:10BE300001DA002B17D0022B06D00020C043F9F7FF
:10BE400069FC1BB0F0BD90E20120F8E7E217521C3C
:10BE500094461A4307D000220892664C62465B1E45
:10BE60001A4307D009E00120FEF7B0FDFEF782FD7E
:10BE70001BB0F0BD0022644C0892674A90427DDD01
:10BE8000664B674A98421FDD914202DC002D05DBBC
:10BE90004DE05848814217DB002D48DD0220FEF7B7
:10BEA00095FDFEF76FFD05460E460022534B2146D9
:10BEB0000898F9F727FB084671004908C00FC0072A
:10BEC000014328461BB0F0BD914215DA002D2EDA51
:10BED0000220FEF77BFDFEF755FD05460E460022CB
:10BEE000464B21460898F9F70DFB72005208C80F1F
:10BEF000C0070243114617E03E4B994223DD002D57
:10BF000015DD0220FEF762FDFEF73CFD05460E46FC
:10BF100000223A4B21460898F9F7F4FA08467100D6
:10BF20004908C00FC007014328461BB0F0BD0220DE
:10BF3000FEF74CFDFEF730FD49004908E20FD2073D
:10BF400011431BB0F0BD002230463946F9F7CCFA58
:10BF5000012205460E46D243F9F7B4FB314A324B73
:10BF6000F9F7C8FA2A463346F9F7CCFA0022284BEB
:10BF7000F9F7C0FA07462A46334600E064E0039129
:10BF800010461946F9F7BEFA3A46039BF9F7BAFA92
:10BF90000746032209915207244B28463146F9F7F8
:10BFA000B1FA07910C90224A204B38460999F9F7CB
:10BFB000A9FA074601911F4A1F4B28463146F9F757
:10BFC000A1FA3A46019BF9F78FFA07460B4602465B
:10BFD000099107990C98F9F7E3F900250E462846D0
:10BFE000079B0C9AF9F780FA3A4627E0FFFF1F00FB
:10BFF000FFFF0F000000F03F0000E0FF0000F07FB7
:10C000000000404301FCFFFF0000F0BF5A0B00009E
:10C010000000E03F0000F0FF0000E0410000F043BE
:10C02000FFFFEF3F555555555555D53F4715F73F40
:10C03000FE822B6544DF5DF80BAE543E099BF9F799
:10C0400059FA02460B4652E1012500202D05A9426E
:10C0500007DA352230463946F9F734FB06463420F4
:10C06000C0430A151218FE48101803900803FD4932
:10C07000000B01430F46FC49884201DC002003E02D
:10C08000FA49884202DA0120119005E0002011905F
:10C090000398401C7F1B039011980597C200F44839
:10C0A0000F927844801843680268394630460D93F1
:10C0B0000292F9F719FA07910C9030460D9B029AFB
:10C0C0000599F9F76DF902460B460020E549F9F7A5
:10C0D00081FA09910490079B0C9AF9F713FA1290D0
:10C0E00000201090E3480D46784400680E9001212E
:10C0F00078104907084311990D9B890440180121C4
:10C10000C90447183946029A0E98F9F7EDF93246F4
:10C11000059BF9F7EFF902460B4629461098F9F707
:10C12000F1F9064602913B4629460E9A1098F9F716
:10C13000E9F9079B0C9AF9F7DDF93246029BF9F70A
:10C14000D3F9099B049AF9F7DDF90591129A0A903F
:10C150002B4610461946F9F7D5F906460246C64859
:10C160000F460B4606217844FEF7A0FB32463B46BD
:10C170000091049010461946F9F7C4F9009B049AFF
:10C18000F9F7C0F906460F462B461946129A109841
:10C19000F9F706F9059B0A9AF9F7B4F932463B46D6
:10C1A000F9F7FEF8109A079104902B4610461946AD
:10C1B000F9F7A8F9B14E0022334609910290F9F738
:10C1C000EFF8079B049AF9F7EBF8002007460246C0
:10C1D00033460091F9F788F9099B029AF9F784F937
:10C1E000079B049AF9F786F906460D913A462946C7
:10C1F000009B1098F9F786F907910C902B46304672
:10C20000129A0D99F9F77EF905460E463A46009BBB
:10C2100005990A98F9F776F933462A46F9F7C0F8EE
:10C2200002460B460746099107990C98F9F7B8F8AA
:10C2300000250E462846079B0C9AF9F755F93A4611
:10C24000099BF9F757F907460722099152078C4BCA
:10C2500031462846F9F756F907910090894A884BEC
:10C2600038460999F9F74EF907460191864A874BF6
:10C2700031462846F9F746F93A46019BF9F790F816
:10C28000834B7B440F9A9B181A685B68F9F788F810
:10C29000029009910398F9F73DFA05910490099BE2
:10C2A000029A07990098F9F77BF87A4B7B440F9A2A
:10C2B0009B181A685B6817460393F9F771F8059B9A
:10C2C000049AF9F76DF80E462846059B049AF9F78B
:10C2D0000BF93A46039BF9F707F9079B009AF9F720
:10C2E00003F9099B029AF9F705F902460B461999D9
:10C2F00000200C900F461898F9F704F90291049069
:10C300003B460C9A19991898F9F7EEF82A463346E5
:10C31000F9F7F8F8029B049AF9F742F809910E90A0
:10C320002A46334639460C98F9F7ECF806460F468C
:10C33000099B0E9AF9F734F8574A0D46914220DBD3
:10C340005242AA18024310D132463B46F9F7CCF8C4
:10C3500004900391514A524B09990E98F9F720F82D
:10C36000039B049AF9F790FA1ED20220FEF72EFBE7
:10C37000FEF708FB49004908E20FD20711431BB042
:10C38000F0BD6A00474B52089A420DD3464AAA189C
:10C39000024300D0CBE532463B46F9F7A5F8099BAE
:10C3A0000E9AF9F771FAF5D96800002340082C4974
:10C3B0000393020D3D4B5218984223DD01200005E6
:10C3C000521CD04042195000400D40183849794461
:10C3D000096813468C463749C1408B43120301213B
:10C3E000120B090551181422101AC1400391002D97
:10C3F00001DA48420390624630463946F9F774F84C
:10C4000006460F4632463B4609990E98F8F7C8FF94
:10C4100000252A46284B28460591F9F773F807911D
:10C420000C90264A264B28460599F9F76BF800919F
:10C43000029032463B4628460599F9F755F8099B84
:10C440000E9AF9F757F81F4A1F4BF9F75BF8009B54
:10C45000029AF8F7A5FF07460B460246099135E018
:10C4600001FCFFFF0000F03F8E9803007AB60B003E
:10C470006A070000AC070000D60600000000084074
:10C4800009C7EE3FFD033ADCF5015B14E02F3EBE29
:10C49000AA0500007005000000009040FE822B6598
:10C4A0004715973C00CC904000346F3F0000E03FC0
:10C4B000C6040000FFFF0F00432EE63F396CA80CB6
:10C4C000615C20BEEF39FAFE422EE63F07990C98D8
:10C4D000F8F766FF05460E46079B0C9AF9F704F835
:10C4E0003A46099BF9F706F809912A4633460E9019
:10C4F00010461946F9F706F8074602462F480B463C
:10C50000059105217844FEF7D1F93A46059BF8F7E5
:10C51000F9FF2A463346F8F7EDFF07460191284612
:10C520003146099B0E9AF8F7EDFF099B0E9AF8F732
:10C5300037FF012304910C9000229B073846019994
:10C54000F8F7D2FF05910E903A4628463146019BF6
:10C55000F8F7D8FF059B0E9AF9F73CF8049B0C9A64
:10C56000F8F7C2FF2A463346F8F7BEFF0022144B05
:10C57000F8F7C0FF064603980D4600054119091556
:10C58000002912DC30462946039AF9F79BF8FEF79A
:10C5900047F9042801D1FEF7FFF930462946039AEE
:10C5A000F9F790F8064601E004E029180B463246F8
:10C5B00021460898F8F7A6FF1BB0F0BD68030000FD
:10C5C0000000F03FF0B58C46002510260521090734
:10C5D0008E620E4C08E067467F5DE760A768FF0744
:10C5E000FCD0E7681F706D1C8542F4DB0020074615
:10C5F00006E0E760A568ED07FCD0E5681D54401C27
:10C600009042F6D38E610020F0BD00000030014062
:10C6100070B572B60124074DA40221462846F9F7E9
:10C620003DFC002804D0224603492846F9F7DAFCED
:10C6300062B670BD00FC0008EC0D0020F8B506469F
:10C640000C46F9F72FFA051E0F4600D001200143D2
:10C6500049000B484908411AC90F0DD0002E01D0DE
:10C66000012100E000210C4361004908401AC00F7D
:10C6700002D10120FEF7AAF928463946F8BD00008C
:10C680000000F07FF8B515460E460746002407E087
:10C690003819C0B200F008F8641C2870E4B26D1CB0
:10C6A000B442F5D33046F8BD10B50446FBF734FF6D
:10C6B000EE20FBF701FFFBF76FFF2046FBF7FCFEC8
:10C6C000FBF76AFFFBF728FFEF20FBF7F5FEFBF710
:10C6D00063FF0020FBF7C0FE0446FBF73BFF20464C
:10C6E00010BD704770B50D460446FBF715FFEE20F0
:10C6F000FBF7E2FEFBF750FF2046FBF7DDFEFBF702
:10C700004BFF2846FBF7D8FEFBF746FFFBF722FF5F
:10C710000A20FEF7A4FA70BDF0B500251026052703
:10C720009C463F070B46BE620C4C06E0595DE1603B
:10C73000A168C907FCD0E1686D1C8542F6DB0020CA
:10C7400007E06146095CE160A168C907FCD0E168C7
:10C75000401C9042F5D3BE610020F0BD0030014086
:10C760000000010203040005405C0000A05C04001E
:10C77000C06C0800805C0400E03F1E00E07D1E00ED
:10C7800007A9022570889B880A0016000100060090
:10C790000100020087008D002D001A3152001A336B
:10C7A0009A001A351D011A376B003B31BE003B332E
:10C7B0005E013B3596023B37000099599959EB5180
:10C7C0008F421E45142E0080EB51F5283333E13A99
:10C7D000703DE13AC235852BC2353333C235C2359F
:10C7E000AE47E13A5138A330513800000000000054
:10C7F00000000102030406070809030406080C10E0
:10C8000018203000000000010203040000000000B6
:10C81000000000000000F03F000000000000F83FB2
:10C8200000000000000000000000004003B8E23FEC
:10C83000000000000000000006D0CF43EBFD4C3E9E
:10C84000033333333333E33FFFAB6FDBB66DDB3F93
:10C850004D268F515555D53F01411DA96074D13FDB
:10C8600065DBC9934A86CD3FEF4E454A287ECA3FD5
:10C870003E5555555555C53F93BDBE166CC166BF57
:10C880002CDE25AF6A56113FF16BD2C541BDBBBE50
:10C89000D0A4BE726937663E0000000000000000B0
:10C8A000C0C8000800000020940100006C5B000874
:10C8B00024C90008940100206C1A0000BCA90008DB
:10C8C0000124130704380D091E0805400826091025
:10C8D0004008560A131D043B08BE0516D8BC40107C
:10C8E000085201033AC842077052030CE5800C1B42
:10C8F0000202DD140901022281F01F668104988979
:10C9000096869679821598039814988796749778E6
:10C9100082439788967197778249F1013D29439226
:04C92000049220005D
:04000005080050C1DE
:00000001FF
